:020000041100E9
:1030000070B501F001F940201F4C0223FE211F4A38
:10301000207401F059F9002821D10223FF211C4A14
:10302000207C01F051F9051E19D1902202211202D3
:10303000207C01F0C3F9032008F07EF880220221F1
:103040005201207C01F0BAF92900207C01F096F9A8
:1030500023681049002B12D001F024F970BDCC2256
:103060003820AC219201207401F0A8F9002802D088
:1030700000232374F0E72368002BEDD106490C22CE
:10308000200007F049FFE7E7FC62FF1F0863FF1F0E
:103090000A63FF1FC0B50011B4B50011F7B5164B98
:1030A0000192C318021D0020009388235B05D318EA
:1030B0001B685C1C1AD09CB2402C18D88D781E0C52
:1030C000AC466746CD782D023D43AE4206D101980D
:1030D00000280ED110000C70240A4C7003249BB2FF
:1030E0000733A343D218009B9A42DED3FEBD44327D
:1030F000F9E71000FAE7C046FC0F0000802213B584
:1031000003000324019189B2520107319B18A143A6
:1031100004305A1A88235B05C3181B68591C03D155
:1031200090429241104016BD99B2402907D80B0039
:103130000733A343C0189042ECD30020F3E7443098
:10314000F9E7134B134A1B68126810B5FA2493422F
:1031500001D81A00F824104BE4021B689A4210D8D8
:1031600013000E4A12689A420ED3013307D1F82396
:10317000DB029C4203D10A49054807F06DFE20009E
:1031800010BDFC24E402ECE7FE24E402F7E7C046AD
:1031900000C0071100D0071100E0071100F007116F
:1031A000FFFFFF7FF0B59BB0150004900391402A0C
:1031B00000D9A0E006AB59801A80FFF7C2FF0400D7
:1031C000042816D9002206A9FFF768FF052810D9A0
:1031D00006AB1B88AB420CD1002D07D0514B2A0007
:1031E0000499C01808F058F8002802D101201BB03B
:1031F000F0BD06AB1D8020000699FFF77FFF041E7F
:103200007BD1069B0793FFF79CFF80235B01C618C9
:10321000802307001B039E4201D3F826F602882371
:103220005B05F31801931B68013302D0019807F086
:10323000A3FE3D49019807F00FFE3B1D0293331D8D
:1032400005938822029B52059B181B6808935A1C01
:103250003CD044219AB20091402A04D80320D11DC9
:10326000814389B2009103991B0C8B4224D0402AE0
:1032700022D80122300008A9FFF710FF021E1BD13F
:10328000380008A9FFF70AFF0400042831D9009A82
:10329000059B9B1880225201B218934240D288238A
:1032A0005B05C118009A09A807F0F6FE1D4B009AAD
:1032B00009A9F01807F038FF009A029B944663446E
:1032C00002931A4B029AFB189A42BAD388235B05E1
:1032D000FC1821680198013907F0BEFD200007F0B5
:1032E0004BFE039A07AB5A8030000799FFF706FFA1
:1032F0000400002C03D1002079E70428FBD988239F
:103300005B05E018069907F0A7FD0323EA1C9A4322
:1033100000D16BE7034B0499E01807F005FF65E760
:103320000424ECE704000011FFFFFF7FF80F00000A
:10333000F7B505001400402A21D8002701AE71809E
:103340003780FFF7FEFE042816D93A003100FFF758
:10335000A5FE042810D93688BC420BD0BD4209D046
:10336000221CB44200D9321C064B92B2C11828006C
:1033700007F092FE30B2FEBDC04300B2FBE703206F
:103380004042F8E70400001137B5042204000D00A4
:1033900001A81649FFF7CCFF020004280BD1019BBE
:1033A000A34208D3AB4204D0104901A80195FFF70E
:1033B000F9FE01203EBD0E4C23682000019307F06A
:1033C000DBFD019920000139019107F045FD8023C3
:1033D0005B01E418074B9C42EED10422034901A88B
:1033E0000195FFF7DFFE0020E4E7C04655550000D9
:1033F00000C007110000081130B589B007F0FCFECD
:10340000102269461E4808F057F81E4B009A9A424F
:1034100005D1019B102B2FD9029B013301D1002331
:103420000293029B002B03D0049304984168084741
:1034300009B030BD10341022200004A908F03CF877
:10344000029B013301D1069B0293882304995B05FB
:10345000C918059B06981A03120B04910592814224
:1034600003D02B4201D107F057FD019B013B019393
:10347000019B002BDED1CFE7E025014C2D03F7E7C0
:103480000000011150485936F7B50F490F4B0A6833
:1034900004001A4084235B0013430B6003000327DE
:1034A0001033019300252E00112007F075FF084B03
:1034B0001B683B40AB4002351E43202DF4D1019BDD
:1034C00040C4A342EED1F7BD5CF0004000FEFEFF19
:1034D00064F00040802270B5AD4CAE4BD2000021AC
:1034E00020001C6007F048FE2300AB4A88331A60B6
:1034F000AA4B1A786E23002A00D01133E3620A2304
:103500002365A74B1878A74BA0630138E361C3B2CA
:10351000032B01D810232362A34B37226361C823F6
:10352000DB00A36123008C331A60082336210F3A95
:10353000E518E16323646264E9670439251DE967DE
:1035400025003B26BC352E602500C0352B602500AC
:10355000C4352A6025000636CC352E602500083E8D
:10356000C8352E602500D03529602100D4310B608C
:103570002100D8310A6021000225E0310D602500CC
:103580004221DC35296025001B3EE4352E602500F4
:10359000E8352B602500EC352A6022000525F43241
:1035A00015602200F0321160220018319032116053
:1035B00022009432136023003C2298331A60AF2318
:1035C000DB002360794B2363032805D807F014FD43
:1035D000330235371523636096232100FA225B00FE
:1035E000A360E360C8332361714BFC319200A36494
:1035F0000A6062626F4A704DA2627322E2656D3AA0
:103600006265A2650232E5644A6002216166962124
:103610008900A166626709210022E166A267674905
:10362000674A684E2167E2673560032811D807F0C2
:10363000E3FC96089EA61023CDE70E23CBE70C23D0
:10364000C9E720001A259C30056020000735A0300E
:1036500005602000A83003602300FA20F8338000C2
:10366000186023006420A433186023005F38AC3353
:10367000186023000338B03318602300C630B43319
:10368000186023000020B833186023003825FC336D
:103690009D604D4D5A665D644C4D9A64DD61962582
:1036A000AD001D624A4D9A675D62F53DFF3D9D622A
:1036B0001E25484ADD6618675867D9651966DA67B6
:1036C000BE23C021444A5B00E250444B4900635092
:1036D00004316250C4225200A350FA23E4205B005C
:1036E0000432A3500432A3503D493E4A3E4BD160C0
:1036F0003E49800019503E49E938FF3819503D498C
:10370000043019503C491038D1613C4911633C499F
:1037100051633C4911603C49195019003B48F8314C
:1037200008603B49D16582213A4A89005A501A0003
:1037300039490832D1671A003849B43211608821FA
:10374000374A89005A501A00364988321160364A81
:10375000DA6407F0B9FD012007F076FC70BD2000A7
:1037600014259C30056020000435A03070E720004F
:1037700010259C30056020000335A03068E720004C
:103780000E259C30056020000235A03060E7C04661
:103790000004FF1FB865FF1FB070FF1F8C45FF1F9F
:1037A0004A0AFF1F3A07000080C3C9019A020000BD
:1037B00050C300006A180000280A0000204E0000D4
:1037C00088130000F009FF1F00400011681000007E
:1037D000C4090000DC05000040420F001027000073
:1037E000FD1BFF1FFC00FF1F0000FF1F252FFF1FF9
:1037F0004D32FF1FE530FF1FD91FFF1FF51FFF1FB1
:10380000A121FF1F491FFF1FC528FF1F8D2CFF1F70
:10381000D918FF1FD127FF1F3925FF1F4525FF1F7F
:10382000491EFF1F011FFF1FC11DFF1FF7B50B0C16
:10383000FF270122009300233C001E001D00944638
:10384000019089B262469A4010000840184136182B
:10385000B6B2FF2F02D1012E00D19FB200980240D4
:103860001A41AD18ADB2FF2C02D1012D00D19CB28E
:103870000133102BE6D10320012E07D1012D04D1F5
:10388000019B2401E4191C700138FEBD102EFCD1EF
:103890000238102DF9D00230F7E710B5064C237826
:1038A000002B07D10548FFF7EFFD0548FFF7ECFDBA
:1038B0000123237010BDC0467865FF1F8C65FF1F74
:1038C0007C65FF1FF0B58BB00D000123019010291E
:1038D00036D8FFF7E2FF00231A001B48C15C013312
:1038E0005218102BFAD1023B002A29D0174B184C42
:1038F0001F68002306A9E25C1600FA5C56405E547D
:103900000133102BF7D102AA07F006FD2A0002A905
:10391000019807F001FB07F01FFC23681B182360C8
:1039200007F01AFC63681B18636007F015FCA368B6
:103930001B18A36007F010FCE3681B18E36000236A
:1039400018000BB0F0BDC0468C65FF1F2C44FF1F54
:103950007C65FF1FF0B5022301245E4E5E4D5F4F74
:1039600033702C703B688FB0552B00D1AEE008202F
:1039700006F01CF8002800D1A8E0002321000093E5
:103980000420574A07F028FB8023DB059C62FFF7E1
:1039900033FD002006F0A2FA07F0DEFAFFF79AFDE9
:1039A00007F0EAFC1F22012400214E4B0EAF1A70D3
:1039B0004D4B1C704D4B19704D4B19689143163A85
:1039C0000A431A60602219689143403A0A431A6018
:1039D00007F052FB07F0A8FAC120FF21454B8000F9
:1039E0001A588A431A50C522920098588843BF3902
:1039F000014399509858404908408021C90101432A
:103A0000802099509958C0050902090A014399502C
:103A100080213A48490107F0A7FB032322003849D7
:103A200001940093374807F01FFC2C22364903A865
:103A300007F032FB03AC61782078023405F0DCFF3C
:103A4000A742F8D10121002006F0C0F80121002092
:103A500006F0ECF80121092006F0E8F82B4B2C4A7F
:103A6000196803201140A022D2020A431A60802262
:103A7000196892040A431A601968264A1140802284
:103A800092030A431A60244B244A934200D801202F
:103A900007F022FC07F018FD07F0AEFC307807F0C5
:103AA000F3FC2878C0B207F06FFA07F0C5FA0C49AA
:103AB000042007F0E1FC06F0DDF900F0A3F800F0C7
:103AC00065FD00F00FFA00200FB0F0BD00233B6051
:103AD0005FE7C0464A0AFF1F8C45FF1F34F00040D5
:103AE0003B000108480AFF1F490AFF1F680AFF1F21
:103AF000BCF0004000E100E0FF00FFFF9045FF1F29
:103B00001458FF1F9055FF1FD8B4001114F0004047
:103B1000FF7FF8FFFFFF9FFFB070FF1F0080FF1FB8
:103B200070B500252849294A29484D6308CA1B0554
:103B30001B0DED188242F9D10022264B8B63264BD8
:103B400008211A628022254B9205DA67244BDA6835
:103B50008A43DA60234A1278012A03D09A682249FC
:103B60000A409A600121EE242048E40002686C4378
:103B70008A430260DA6811208A43DA6007F0C4FBE6
:103B8000112007F0E9FB112007F096FA184A200CE3
:103B90000400642390420AD8FA220023D200904203
:103BA00005D9144B0A21C01807F05EF9C3B2124AB6
:103BB0001372124BD4801B78002B04D1104B1021B0
:103BC000187807F059F970BD0000054088050540D8
:103BD00000060540FF01000000F0004004E100E0A5
:103BE0003CF000404A0AFF1FFFDFFFFF00380040A3
:103BF000B70B000030F8FFFF1063FF1F3265FF1F97
:103C00002863FF1F002210B51100112007F004FCEB
:103C100010BD0000F8B5002301250826394F3A4CA5
:103C20003B62E3681120AB43E360E368B343E360C6
:103C300007F092FB112007F067FB112007F0F4F961
:103C40004023226829001343236080236268DB023B
:103C5000134380226360A36807201343A360A36813
:103C60002A4A1340A3608023A2689B0113431022B9
:103C7000A360236C93432364236C2B43236480232E
:103C80005B003B62226B224B1A402263626B1A403C
:103C90006263A26B1A40A263E26B1340E3631D4AA6
:103CA000E3681340E36005F091FF2900072005F069
:103CB000BDFF8021184A1120536C0B43536407F059
:103CC000C3FBFD21154B164A89005A508023C7209B
:103CD000626B5B0313436363E36880003343E36019
:103CE000E368104A1D43104BE560195811408022CB
:103CF00012020A431A50802292051A600B4B5E632F
:103D0000F8BDC04600F000403CF00040FFFFDFFF80
:103D1000EFFFEFFFFFFF7FFF003800400000FF1FB5
:103D2000213B0011FF00FFFF00E100E00000054023
:103D300030B503A804880B20002C0ED14968074D2C
:103D400008784978090201430A20A94205D10121D6
:103D500020001980024B1B7A137030BD192A000015
:103D60001063FF1FF7B5150008AA16884A680F4FA1
:103D700014785278120222430A24BA4214D1012242
:103D8000DBB2019200962A0006F0C4FF041E0BD19C
:103D9000074B1B68002B07D068782A780002104375
:103DA00042425041013098472000FEBD02290000E8
:103DB0009462FF1F30B5012503790400BFB02B4288
:103DC00012D00A49408806F011FB28420CD06A46FE
:103DD000074B69465B8D55801380064B60881B7AC4
:103DE0001371002203F0C4FB3FB030BD8C62FF1F93
:103DF000D041FF1F1063FF1F10B50549054806F0AD
:103E0000ABFA0421044A054806F068FA10BDC04622
:103E10008C62FF1FFFFF000004B50011D041FF1F9F
:103E200010B5024804F02AFA10BDC046B53D001195
:103E30000623837010330371443B43712A3383712B
:103E40004433C37100230222012110B503720E4BCB
:103E5000027041701C8881724472197A0273C172B7
:103E60009A784273DA7882730322C2731A790274E1
:103E70005A7942740C2282749A79C274DB79037580
:103E80001123C37010BDC0461063FF1F10B514206E
:103E900007F01AF9124B14220021186007F084F879
:103EA000002007F079F9012007F04EFA022007F010
:103EB0001BFA032003F086FC042005F09BFC052080
:103EC00002F0D4FE062003F091FB072000F03EFF35
:103ED000082006F0E3F9092000F042FD10BDC046BD
:103EE0009862FF1F10B507F0D7FA012007F0BCFA5F
:103EF00007F06AF8002010BDF7B50E00377A1C00F5
:103F000008AB11003D001A8820231D401F423DD1FF
:103F10003378022B3CD173681F785B781B023B43DC
:103F20001E4FBB4208D01E4FBB4217D01D4DAB42A7
:103F300022D00A252800FEBD002A2BD1142C2BD814
:103F40002200F06806F0E8FF174B1C70012CF1D935
:103F50004021164B187806F08FFFEBE7002A19D1A5
:103F6000202C19D82200F06806F0D6FF104B04214F
:103F70001C700E4B1878EEE7E3B201240092019416
:103F80000A00310006F0C6FE0500D3E70825D1E798
:103F90000125CFE70B25CDE70D25CBE7F3FF00008B
:103FA000F4FF000002290000C662FF1F2863FF1F04
:103FB0009C62FF1F094B10B50400984205D00129EF
:103FC00004D12000064906F0C7F910BD0229FCD132
:103FD000013904F011F90028F3D0F6E7FEFF0000E4
:103FE000BE62FF1F70B50D7A100004AA2C0016885F
:103FF00010221440154220D1002E20D10A78022A26
:1040000018D14A68517815780E4A0902294391421D
:1040100005D00D4A914209D01C800A2404E01422E4
:104020000A491A8006F078FF200070BD0C2208496A
:104030001A80F7E71C800124F6E70824F4E70B2434
:10404000F2E7C046F3FF0000F4FF00001044FF1F3A
:104050001C63FF1F10B504000749084806F07CF9EF
:10406000074804F04BF80020E40704D50721054A6F
:10407000054806F033F910BDBE62FF1FFFFF0000C8
:10408000B53F001148B500111442FF1F00B5BFB085
:104090006A460B4B0B491B8801A813800A4B1A7800
:1040A00000F0A8FA6B4680B25880002805D0074B74
:1040B00000226946188803F05BFA3FB000BDC04695
:1040C0006E42FF1F9D62FF1F9C62FF1F7043FF1F18
:1040D00000B5BFB06A460B4B0B495B8D01A813803E
:1040E0000A4B1A7801F0ACF96B4680B25880002870
:1040F00005D0074B00226946188803F039FA3FB013
:1041000000BDC0461442FF1FC762FF1FC662FF1FEB
:104110007043FF1F70B5160004AA148805AA15780D
:104120004A685078117800022A4A08438018052806
:104130004BD806F061FF03131E29343F0720042CDF
:104140000BD80522121BAA4200D92A0022491A8044
:104150003000091906F0E0FE002070BD0720132C86
:10416000FBD81422121BAA4200D92A001B491A802C
:10417000EEE707200E2CF0D80F22121BAA4200D91E
:104180002A0017491A80E3E70720032CE5D8042208
:10419000121BAA4200D92A0012491A80D8E7072028
:1041A000032CDAD80422121BAA4200D92A000E4995
:1041B0001A80CDE70720032CCFD80422121BAA4275
:1041C00000D92A0009491A80C2E700220A201A8071
:1041D000C3E7C046DCD5FFFF93B50011E462FF1FC3
:1041E00083B500117EB5001179B5001174B50011C9
:1041F00010B50D21024A034806F070F810BDC04604
:1042000068B500118442FF1F10B50021162005F08B
:1042100049FD0121152005F045FD07F0A5F8040032
:10422000092006F001FF0022184BDA6661321A609D
:1042300019685B3A9143023A0A431A60144A94425D
:1042400009D10A22DA6107321A6200221A639A63DC
:104250000132DA6310BD0F4A944203D11E22DA61A3
:104260000532F1E70C4A944203D13022DA6106327A
:10427000EAE70A4A944203D14322DA610832E3E7CB
:10428000074A9442E1D16922F7E7C0460050004056
:104290000024F4000048E801006CDC020090D00328
:1042A00000D8B80510B50024064B0920DC6607F0DD
:1042B00053F82100162005F089FC2100152005F097
:1042C00085FC10BD00500040F8B51C000023134DC4
:1042D0000F00EB666860160006F08EFF0123802257
:1042E000EB6623002F615200013B08D206F00CFE62
:1042F00008200B4A1168002C03D12000F8BD2A6168
:10430000F2E72B6F034203D02B69013C3370013677
:1043100013685B1A012BEED90124EEE70050004030
:104320006008FF1F002370B5124D1400EB66686033
:104330000E0006F061FF01238022EB66230052008D
:10434000013B08D206F0E0FD08200B4A1168002C62
:1043500003D1200070BD2A61F2E72B6F034203D026
:104360002B69013C3370013613685B1A012BEED9BF
:104370000124EEE7005000406008FF1F002370B5E5
:104380000C4C0D00E366606006F036FF0123E36627
:10439000256106F0B9FD8020074A80001168636B33
:1043A000034205D113685B1A012BF8D9012070BDB7
:1043B0000020FCE7005000406008FF1F002370B59C
:1043C000134C0E00E3666060150006F015FF012334
:1043D000E36626610F33626B1A42FCD02B0A23611D
:1043E0001023626B1A42FCD0EDB2256106F08CFD01
:1043F0008020084A80001168636B034205D113686E
:104400005B1A012BF8D9012070BD0020FCE7C046E3
:10441000005000406008FF1F13B5344C237C002B74
:104420005FD0FFF7F1FE207C38283FD10722694694
:10443000FFF778FF002854D16B461B787F2B50D8AC
:10444000CC22AC219201207CFFF7B8FFFFF72AFFB6
:104450006B46D878F02302041B031A406B469B88F6
:1044600023495BBA9BB21A4323680009534322894C
:104470001B0C9B184B806B465A789B7812031B01D0
:104480001A4302436368534362891B0C9B181BB297
:104490008B80002B04DA0022154B9A80002016BD79
:1044A000144A9342FADD124B124AF6E76946042297
:1044B000FFF738FF011E14D1207CFFF75FFFFFF7E5
:1044C000F1FE6B461A88236852BA92B2534322898E
:1044D00007491B0C9B184B806B465A8852BA92B204
:1044E000D0E7FEF78DFD0120D9E7C046FC62FF1F33
:1044F0001063FF1F0F27000010B51B4B1A793F2ACE
:1045000001D93F221A711979184A194811701822D5
:104510001849028018480A8002804A809A79174810
:10452000802402800C208A80013242432401101C26
:10453000A24200D9201C124AC88010805A79002A51
:1045400001D101325A711A7A002A01D101321A724C
:104550005A791B7A0B4853430A21584306F084FCCE
:10456000094C206010BDC0461C63FF1F480AFF1F96
:104570006E43FF1F3845FF1F6C43FF1F6A43FF1F39
:104580006843FF1F710200002C63FF1F10B5062156
:104590000020FEF7F9FE124C002807D10C22200063
:1045A000104906F0B9FCFFF7A7FF10BD0C22200050
:1045B0000D49FEF7BDFE0C2804D00C22200009494D
:1045C00006F0AAFC094C0C2220000949FEF7B0FEB7
:1045D0000C28E8D00C220021200006F0E5FCE2E7E0
:1045E0001C63FF1FCCB50011FC0C0000FC62FF1F18
:1045F000F50C0000F7B5040000200D000100824218
:104600000CD02B7860702370834208D10123637033
:10461000133363800E3BA06063600C30FEBD552BEE
:1046200019D1013A624E0C2A13D8002A0AD0691C0B
:10463000300006F071FCFFF75FFF0C2230005D498F
:10464000FEF7B0FD0C223100601C06F065FC0D2069
:10465000E4E70C22EBE7562B10D1554D0C225649BE
:10466000280006F059FCFFF747FF0C2251492800AB
:10467000FEF798FD0C222900601CE6E7252B17D1D8
:10468000013A4E4E0C2A11D8002A08D0691C30007D
:1046900006F042FC0C2230004949FEF783FD11224E
:1046A0003100601C06F038FC1220B7E70C22EDE761
:1046B000262B0AD1414D1122280006F075FCFEF789
:1046C0009FFC11222900601CECE7DC2B1DD1022A83
:1046D0006BD96B786370AB78A3706E781B021E4346
:1046E000032A05D0033A310092B2E81CFEF75AFDC6
:1046F00010223100E01CFEF71BFE03000330002BEC
:1047000000DB8BE70220637088E7DB2B20D1042AD3
:104710004BD9A9786B7809021943EB782F791B04E0
:104720000B433F0610261F43052A05D0561F3200B3
:104730003800691D06F0F0FB05222900200006F074
:10474000EBFB32003900601D06F0E6FB701D65E7EB
:10475000DA2B2AD1042A28D9AB7869781B020B43BB
:10476000E978090419432B791B060B43082A19D948
:10477000AA79697912020A43E979090411432A7A6C
:1047800012060A4301921A601B68052229002000C4
:10479000019306F0C1FB0422601D01A906F0BCFBD9
:1047A00009203BE7FE226270EEE7FF23AAE7C0463E
:1047B0001C63FF1FFC0C0000CCB50011FC62FF1F46
:1047C000F50C000070470000013870B5042809D8C6
:1047D00006F012FC030921081200144B022118787C
:1047E00006F04AFB70BD114B0821187806F0DCFD7D
:1047F00000220F4B1A71F5E700240D4B0B4D0821D9
:1048000028781A681C719C7106F006FC2100287833
:1048100006F0FAFCE6E70123054C0821A371034BDF
:10482000187806F0C1FD00232371DBE72863FF1F22
:104830002C63FF1F10B5002903D10920013105F0B9
:10484000F5F910BD10B5084B084C9881D881188235
:104850005882207802F0A8F80422054B0121207824
:104860001A7006F009FB10BD3644FF1F6265FF1F7A
:104870006165FF1F10B501290DD11322064B0021E0
:1048800009209A7105F0D2F9044B1B78002B02D055
:104890000348FFF7D7FF10BD2C63FF1F3265FF1FD2
:1048A000C40900000300F0B50A4D8E18B14202D1D0
:1048B00052008018F0BD0C782F6824093C5D0F274A
:1048C0001C700C7801313C402F683C5D5C700233F9
:1048D000ECE7C0466443FF1F10B50A4A0A490820A6
:1048E00005F0A6FA092005F08DFA0121092005F04E
:1048F0009DF9002005F086FA0121002005F096F9C7
:1049000010BDC046354800117548001110B5114B57
:104910001A781870002A0ED000280BD10E4B1A7886
:10492000062A07D85423D340DB0703D50B4B18784E
:1049300002F03AF810BD0028FCD0074B1B78012B81
:1049400002D0033B022BF5D8044B0121187806F066
:1049500093FAEFE73265FF1F6165FF1F6265FF1F76
:10496000F0B5554D85B02870FFF7B6FFFEF748FB50
:1049700006F0E2FA002002A90290039006F064FC1F
:1049800003224E494E48FFF78DFF2D2403000422D9
:104990001C704C490130FFF785FF0222047002A908
:1049A0000130FFF77FFF0222474B484CDA87200097
:1049B00006F00AFD022815D0062220004449FEF721
:1049C000B7FC06280ED00321200006F035FA8D230F
:1049D000E3706E3B23710622193320003C4963715A
:1049E000FEF7E0FB0E233B4F3B4C3C4E3B70013B44
:1049F00023700522043B300039496370019606F0AC
:104A00008BFA2D23012237493748E371FFF74AFF1C
:104A100001223649FFF746FF01222C49FFF742FFEA
:104A20000020FFF773FF324E324A0121324B1278D9
:104A3000307801F07BFF3A7801272300002130789D
:104A400001F074FF21782D4B0139019AC9B2002081
:104A50001F7005F061FBFA221B4B52019A81DA812B
:104A60001A825A822021287806F06EFA01204042EC
:104A700005F09EFB0120404205F03AFCFFF7B8FB31
:104A8000FFF7BAF900F074FC01204042FFF7E2FAA8
:104A9000380006F001FAF72001F004F9390028780F
:104AA00006F0EAF9287802F0DBF8154806F0D4FAA7
:104AB000FFF7B0F805B0F0BD2863FF1FAC44FF1F3F
:104AC000E462FF1F0863FF1F3644FF1F6509FF1FD5
:104AD000ADAC00002E65FF1F0F65FF1F1165FF1FA6
:104AE00093B500116709FF1F1765FF1F6609FF1FB8
:104AF0006265FF1F9843FF1F7943FF1F0065FF1F7B
:104B00003463FF1FF8B50A0020230D001A40194234
:104B100032D0444B1B78002B2BD0434C434E23798F
:104B20000133DBB22371327A9A4215D800272771FC
:104B3000FFF772FC63790133DBB26371727A9A42D8
:104B400002D86771FFF766F8394F3800FFF770F940
:104B50003900152006F048FCA379002B09D0013B51
:104B6000DBB2A371002B04D1707964335843FFF793
:104B700069FE20206840F8BD0BB2002B0ADA2D4BED
:104B8000187806F0A1F9002801D006F075FB802006
:104B90000002EFE702240E002640214206D0224BFD
:104BA00001201A71FFF7B2FE2000E3E70B0711D5D1
:104BB000FFF732FC00F0F6FB1B4A1C495379013326
:104BC000DBB25371497A994202D85671FFF722F845
:104BD0000820CFE710240E002640214206D0114BBA
:104BE0001B78002BE0D1FFF71BF9DDE70124214200
:104BF00009D0114800F06EF806F0D6FA310009200D
:104C000005F014F8D0E70424214202D0FFF73EFA61
:104C1000CAE74024080020402142ACD0FFF758FAF0
:104C2000C2E7C0463265FF1F2C63FF1F1C63FF1FD6
:104C30007943FF1F2863FF1F5C43FF1FF0B51B4B29
:104C40001B4F1B883A8804001A4E1B4D85B09A42B0
:104C50000DD832889A420AD3184B1A882B889A4268
:104C600005D1174A174B12881B889A421BD0052082
:104C700001F06EF83B8802AA1380338801905380BC
:104C80002B88114D93800F4B02A91B88D3800F4BAB
:104C90002A78188802F07AFD0D4B08212878019AAD
:104CA0001C7006F001FB05B0F0BDC046FE64FF1F9E
:104CB0006E43FF1F6C43FF1F6A43FF1FFC64FF1F0F
:104CC000FA64FF1F6843FF1F6265FF1F7043FF1FE9
:104CD000F864FF1F13B50C4B1C78002C11D1002871
:104CE00001D00A4B18600A4A0A4B11780A4A107818
:104CF0000A4A01920A4A0092002205F005F92000B2
:104D000016BD1124FBE7C0466165FF1FF464FF1F59
:104D10006065FF1F5065FF1F6265FF1F3C65FF1F39
:104D20004065FF1F10B5064B12201B78052B06D1DE
:104D3000044B13221988044B187801F0E5F910BDD3
:104D40006165FF1F7043FF1F6265FF1F10B50024E0
:104D50000122114B52421870104B1C70104B1A80DC
:104D600001F07EFF04220F4B21001A700E480C3216
:104D700006F01AF9102221000C4806F015F9072256
:104D80000B4B1C600B4B1C700B4B1C700B4B1A70AD
:104D90000B4B1C7010BDC0466265FF1F6165FF1F95
:104DA0007043FF1F6065FF1F5065FF1F4065FF1FB9
:104DB0003C65FF1F0E65FF1F0D65FF1F7243FF1F40
:104DC0000C65FF1FF8B5174C0600257806A81424BB
:104DD0000078052D23D1B41F134FA5B21824BD426E
:104DE0001DD88D1FADB2BD4219D8FA256D00AA425B
:104DF00015D21D000D4F0A3DADB2BD420FD80C4C6F
:104E000026800C4C21800C4900240A800B4A138018
:104E1000FFF714FF0A4B0421187806F0C5FA2000AA
:104E2000F8BDC0466165FF1F790C0000750C0000DD
:104E30006E43FF1F6C43FF1F6A43FF1F6843FF1F42
:104E40006265FF1FF0B50BB20D0089B0002B00DBCF
:104E500076E1A64E307806F037F8041E55D0037878
:104E6000A22B00D127E1D02B1AD0912B4AD1437825
:104E70000E2B47D19E4B82889A4243D19D4A83682C
:104E80001278052A3ED1032018567F283AD09A4B33
:104E90001B68002B36D05B68002B33D0984731E07D
:104EA000807807282ED806F0A7F8042D1D444479F1
:104EB000ADDD6378002B11D10622E11C8F4806F08E
:104EC0002BF801218B4B19708D4B1A78002A5BD07F
:104ED0008C4B307801F02AFD002855D00722854BF5
:104EE0001A7051E061780029F8D1E378002B11D0D5
:104EF000854A864B1278307801F018FD607063782F
:104F0000002BEBD1200006F0B7F9802000026840AA
:104F100009B0F0BD774B1B78022BF3D0012130781C
:104F200005F0CAFF0028EAD10121307805F0A4FF7E
:104F3000E5E76378002BD1D16E4F032807D13B788A
:104F4000052B02D101333B701EE00223FBE7704BBF
:104F50001A88704B0293002A0BD01B78002B03D0C9
:104F60000121307806F0A0F93B78062B04D1013BF3
:104F7000E9E7029B1A70F7E7042B41D10121029B5C
:104F80003078197005F078FF5B4B1B68002BB9D0A7
:104F90001B68002BB6D0574A10787FE76378554FCF
:104FA000002B27D10622211D5B4805F0B5FF628941
:104FB0005A4B5B491A80A2895A4B1A80E3890B80AD
:104FC0000521397058490A80584A1380228A584B63
:104FD0001A80584B1B78012B09D11F2000F0B8FE16
:104FE000FA22920042430421307806F05DF9002253
:104FF000484B75E7312B00D070E70022454B1A7003
:105000000323A0E706220021434805F0CDFF00233B
:10501000454A04211380454A30781380444A13805E
:1050200006F0C2F90821307806F0BEF9A379083BF2
:105030005A4253412F4A03331370314B1B78002BD4
:1050400006D0344B30781A78002A06D001F0ACFC38
:105050000122324B52421A8096E70121197005F065
:105060000BFFF5E70821307806F09EF96378002BF6
:1050700000D047E72C4B2E4F0293E388029A04217D
:1050800013802A4B307803932389039A1380638912
:105090003B8005F011FF002800D033E7264B1B684A
:1050A000002B00D12EE7039902983A8809880088DE
:1050B0001B68984726E74379132B00D022E7038922
:1050C000012B0AD11D4B1B78022B06D10821307809
:1050D00006F06AF9FFF726FE14E7052000F038FE17
:1050E00008210200307806F0DFF80BE76265FF1F49
:1050F000051400006165FF1FF464FF1F3365FF1F87
:105100009843FF1F7943FF1F2E65FF1F0F65FF1F89
:105110003065FF1F3265FF1F0165FF1F7043FF1FD2
:105120000865FF1F0A65FF1FFE64FF1FFC64FF1F69
:10513000FA64FF1F0065FF1FF064FF1FF864FF1F84
:105140008020C001014200D0E1E6CB0731D5324BCF
:105150001B78002B1DD0314E05AC3378052B1AD1AE
:10516000023B23702E4B21001B7823722D4B1B78A2
:1051700063722D4B187801F07DFB002809D00720C1
:105180002A4B30701B68002B03D01B68002B00D00B
:1051900098470120BBE60E20254B06221B782549A7
:1051A0002370254B1B78637002ABC01805F0B4FE6A
:1051B000D8E7022308001840194209D0174B1B7882
:1051C000052B03D11D4B188806F0DEF802209EE661
:1051D0000424214203D0FFF731FD200097E6082385
:1051E00008001840194200D192E6154B1C78012C9A
:1051F00003D0022C0DD0082089E6124B124A134925
:1052000013481B881288098800880094FFF7DAFD8C
:10521000F1E7FFF787FDEEE73265FF1F6165FF1FCE
:105220007243FF1F0C65FF1F6265FF1FF464FF1FC1
:105230000E65FF1F7343FF1F0D65FF1F7043FF1FA8
:10524000F864FF1F6843FF1F6A43FF1F6C43FF1F83
:105250006E43FF1F10B502A804880B20002C10D14C
:10526000496808784978090201430C48814209D10C
:10527000022119800A4B59881170DB7800205BB23B
:10528000537010BD074C0A20A142FAD102211980A7
:10529000034B998811705B79F0E7C0466E2A0000D5
:1052A0001063FF1F6F2A0000F7B5150008AA1688C3
:1052B0004A680F4F14785278120222430A24BA42E5
:1052C00014D10122DBB2019200962A0005F022FDE2
:1052D000041E0BD1074B1B68002B07D068782A7877
:1052E0000002104342425041013098472000FEBD69
:1052F000022900007465FF1F30B501250379040001
:10530000BFB02B4227D01549408805F06FF82842DE
:105310000DD06A46124B69465B8D13800223538081
:10532000104B5B8893806088002202F021F90E49BF
:10533000608805F05BF8C0070DD56A460B4B6946DF
:105340001B88138002235380064B9B8893806088C0
:10535000002202F00DF93FB030BDC0466C65FF1F62
:105360009C43FF1F1063FF1F6465FF1FF643FF1F71
:1053700010B5074C0749200004F0EEFF2000064955
:1053800004F0EAFF0721054A054804F0A7FF10BD15
:10539000FFFF00006C65FF1F6465FF1F4CB6001126
:1053A0009C43FF1F10B5024802F068FF10BDC046C5
:1053B000F95200110200F0B501270A480A4E5118AF
:1053C0008B1A002B00DCF0BD0824157843086840D8
:1053D00038404000805B013C58406D08002CF5D1FE
:1053E0000132EDE7FFFF000066B60011F0B50025C1
:1053F0000F269D4200DBF0BD4C5D07094440344060
:10540000A400A05801357840F3E70000F0B589B05A
:105410006A460D000B000F27110010351C78013370
:10542000260024093E40167054700232AB42F5D17A
:105430002023024AFFF7DAFF09B0F0BD6CB6001175
:10544000F0B54E780B7889B036020D001700019048
:105450001E43012A5AD98E4B9E4200D871E0013377
:105460009E421CD1062A17D1CA788B7812021A43A1
:105470000B791B0413434A7912061A43854B5A6170
:1054800000221A705A80844A5A60844A9A60844A78
:10549000DA60002009B0F0BD88225205EEE7814BAA
:1054A0009E4235D17B498B78002B00D0E8E00C2A56
:1054B0002AD10F22AB789343EA78120213432A7958
:1054C000120413436A79120613434B60EA79A879F0
:1054D00012020243287A000410436A7A1206024339
:1054E000CA60EA7AA87A120202436F484A8183426C
:1054F00000D8C7E01201D21889235B059A4200D96F
:10550000C0E001238B70C4E7022AFAD00523A5E08E
:10551000664A0123964200D0A0E0FFF703FC052F66
:105520000CD9EB78AA781B0213432A7912041A4388
:105530006B791B0613435E4A0393136005F0DCFC92
:10554000A7E7544C2378002BA3D1A378002B00D1DC
:105550009AE02289531C9BB29E4200D08BE0132F0D
:10556000D4D9CF7C8B7C3F02122128001F43FFF748
:1055700021FFB84200D089E0002E3BD1EB78AA7819
:105580001B0213432A7912041A436B791B06134337
:10559000E26803939A4260D1FF23AB70EB702B71EA
:1055A0006B716389002B16D0606837013818000BC7
:1055B000636900030390984205D9606105F0DCFC43
:1055C000E3780133E37060681022A91C381805F0F5
:1055D000ABFD26815DE7EB7B2A7C1B0212041343A3
:1055E000AA7B134303931B09013363816389B3428D
:1055F000DAD832E067897B1E9BB29E42F6D1EB7807
:10560000AA781B0213432A792A4E12041A436B7993
:1056100065681B0613433100042204A8039305F0B8
:105620007BFC291D0C2205A805F076FC012004A9AD
:1056300040421035FFF7EAFE013F012F16D1039BD0
:105640002061834209D104223100606805F06CFDBD
:105650000422606803A905F0E7FD09230D4914221F
:1056600001980B7005F058FC142013E72900FFF790
:10567000CDFE1035E0E70723964200D809E7EDE7B5
:105680000223EBE70423E9E70323E7E70623E5E743
:10569000FFFE00001044FF1F00000111FFFF00008B
:1056A0005048593601FF0000FFFF001102FF0000C3
:1056B00034F000401C44FF1F10B5034C0B000122C6
:1056C000210000F06BFA10BD795800110B8870B5FD
:1056D00006000D000224162B11D92B0003220949C4
:1056E00000F05CFA041E0AD1074B2A881B88191C9B
:1056F000934200D9111C300089B200F0EFFA20006B
:1057000070BDC046A5580011D265FF1F10B54A787C
:105710000400013A0B000220012A07D80A78002A67
:1057200004D005222000024900F038FA10BDC0461E
:10573000D35800110A7810B50B0004000220002A8B
:1057400004D007222000024900F028FA10BDC0460C
:105750007F5900110A7810B50B0004000220002ABE
:1057600004D009222000024900F018FA10BDC046FA
:10577000E559001110B5034C0B000B22210000F07D
:105780000DFA10BD155A001110B5034C0B000D2277
:10579000210000F003FA10BD875A001110B5034C28
:1057A0000B000F22210000F0F9F910BDE15A0011A1
:1057B0000A7810B50B0004000220002A04D0112240
:1057C0002000024900F0EAF910BDC046F15A00116C
:1057D000002310B51322190000F0E0F910BD0000FD
:1057E00010B5034C0B001722210000F0D7F910BDB3
:1057F000435B0011002310B51922190000F0CEF907
:1058000010BD000010B5034C0B001B22210000F05E
:10581000C5F910BD7D5B0011F7B584890D00060048
:105820000121002C22D000238268D3561778002B48
:105830001EDA0C2C1AD90C3CA4B213194088009320
:10584000230002F076FE431E984101307B06DB0FF9
:105850006B703F23013C1F40A4B22870AF70AC8036
:10586000002C07D0B3680133AB6000210800FEBDF7
:105870000020EBE7AC60F8E70B7803704B884370CF
:105880004B881B0A83700B79C37004207047042077
:10589000022B06D10020537811781B02009A0B438B
:1058A000138070470B8803700B881B0A437002201B
:1058B00070470420009983420AD1537810781B0264
:1058C00003430B80D37890781B02034300204B8066
:1058D0007047F8B50D004B7801240021461C037079
:1058E0002B788B4201D82000F8BD6B78B01C4F1C80
:1058F000012B10D1890069184B88022233704B8824
:10590000B9001B0A7370691805F006FB04360434ED
:10591000A4B2F9B2E4E7122359436B185A88043150
:1059200032705B8810221B0A7370691805F0F4FA54
:1059300012361234ECE770B5049D14001E00052BDE
:1059400001D8042070BD637812781B0213432B80AA
:10595000E378A2781B02134302226B802A71211D77
:10596000681D063E05F0D8FAB2B22A81F02AE8D8BE
:105970002800A11D0A3005F0CFFA0020E2E700233D
:1059800010B50A789A4201D8900010BD9A008A1882
:105990005488013304705488DBB2240A447094881C
:1059A00084709288120AC2700430EAE710B51100C0
:1059B000029C062B04D004201022142B01D010BD11
:1059C000022222714B7808781B0203432380CB7894
:1059D00088781B02034363800431601D05F09CFA44
:1059E0000020ECE710B50C788B7804315C43E4B20E
:1059F00003702200013005F08FFA601C10BD0420F6
:105A0000022B06D10020537811781B02009A0B4319
:105A10001380704710B50C000A88023105F07CFA3B
:105A2000208810BD70B504000D0004981100012BF2
:105A300001D8042070BD16785278120232430280D9
:105A40000200F83255701470E825002C00D10C3596
:105A5000023B9AB24280AA42EBD80231043005F0F0
:105A60005BFA0020E6E70420009983420AD15378CC
:105A700010781B0203430B80D37890781B020343FA
:105A800000204B80704710B50C000A88023105F0E9
:105A900043FA208810BD000070B501211E000420CB
:105AA000049C0E400B4218D1CB40DDB28D4214D97C
:105AB0000A49DBB2098899420FD32300F6331D70DF
:105AC0003300580011184978165C0902314301333C
:105AD0002152D9B28D42F4D8002070BD3044FF1F4E
:105AE00010B50C000A88023105F016FA208810BDA6
:105AF00010B50C788B7804315C43E4B2037022005B
:105B0000013005F009FA601C10BD10B511000298B3
:105B1000032B01D8042010BD14785278043B1202E4
:105B200022430280CA788C781202224342809AB2C1
:105B30008280F22AEED80431063005F0EDF900201B
:105B4000E9E710B50C000B8803700B881B0A437043
:105B50004B8883704B881B0AC3708A8804300631D7
:105B600005F0DAF9A088043080B210BD0420012BC2
:105B700003D100201378009A1370704710B50C0001
:105B80000B8803700B881B0A43704A88023004316B
:105B900005F0C2F96088023080B210BDF0B589B05E
:105BA00003931E4B029242000700D05A019102F06B
:105BB00010F81325061E2DD0029B01240370019BB3
:105BC000002B04D0001903999847001984B26B4642
:105BD0001B7A5BB2002B0FDA1021380002F00CFBAD
:105BE0001925002813D130003219E1B202F056FC19
:105BF000051E0CD10C34A4B2042304AA380005A954
:105C000093800696948101F09FFD051E02D030001E
:105C100005F03AF9280009B0F0BDC046D065FF1F75
:105C200070B505000C0000280CD00020814209D07E
:105C300010222000044905F06FF901202B7823730E
:105C40006B78637370BDC046ACB60011F0B506004A
:105C50000D0017001C0085B002291BD00020102960
:105C600007D1022B07D0102B03D115E00020102CF8
:105C700008D005B0F0BD69463800FFF7D1FF2A0013
:105C800069460BE069463000FFF7CAFF220069460B
:105C9000380004E0022BE9D12A003900300005F079
:105CA000B3F9E6E7031CF72800D9F72303200849D6
:105CB0009AB2013A0B80D317034006499B189B10F8
:105CC0000B80D30F04499B185B100B807047C046B4
:105CD0003444FF1F3244FF1F3044FF1F034B1B8817
:105CE0008B4202D3024B4000C15270473444FF1F25
:105CF000D065FF1F014B4000185A7047D065FF1F49
:105D00001722014B1A807047D065FF1F70B5050040
:105D10000E2005F041F9041E13D0D0230370002398
:105D20000622837007494570033005F0F5F8064BED
:105D30002100DA8A62811B7E2373044B187805F0F8
:105D4000BBFA70BDEC65FF1FDC65FF1F8444FF1FBD
:105D5000262803D8024B4000C05A70470148FCE790
:105D60003644FF1FFFFF000070B506000C00094D10
:105D70001C220021280005F017F9074B1E70074B65
:105D80001C7005F0D9FA0123002801D0002312204D
:105D90002B7070BDDC65FF1F8444FF1FFD65FF1F76
:105DA00070B505000D4C0800E260A16010220021D2
:105DB000656005F079F9012803D11021A06802F08F
:105DC00048FD10220021280005F06EF9012803D1BA
:105DD0001021606802F03DFD70BDC046DC65FF1F0C
:105DE00070B5041E05D1002903D006220D4805F028
:105DF00093F80D4B1D78012D11D1002C05D10222F5
:105E00001A7005F011FB280070BD00221A70074BB4
:105E10001B78FF2BF7D02000FFF778FFF3E7002572
:105E2000F1E7C046EC65FF1FDC65FF1F8444FF1FE0
:105E3000030010B5002801D1002010BD00780B4AE6
:105E4000002803D15988D1821B7913761378022B4D
:105E5000F2D10023984200D103331370044B1B7816
:105E6000FF2B01D0FFF752FF0120E6E7DC65FF1FA3
:105E70008444FF1F002911D000280CD04B79012841
:105E800003D140225242134303E03F221340032830
:105E900002D001204B7170474022F4E70800FAE776
:105EA00070B5094D0100287800280BD0074C062258
:105EB000200005F031F821002878FFF7DBFF2000F3
:105EC00005F07AF870BDC046FC65FF1FD665FF1F60
:105ED00000290AD0012808D13F224B799343C02BD7
:105EE00003D0403B5A425341981C704770B5174D40
:105EF00006002B78FF2B15D00A2005F04DF8041E64
:105F000010D0D0230370C83B8370114B11491B780C
:105F10004670C3700622043004F0FEFF210028788A
:105F200005F0CAF90C4B1B78012B0DD10B4B1B68EC
:105F3000002B03D09B68002B00D09847084B04210E
:105F40001878084A05F068F870BDC0468444FF1F01
:105F5000FC65FF1FD665FF1FF865FF1F2466FF1F46
:105F60002866FF1F60EA0000014B98687047C04632
:105F7000DC65FF1F014BDB6818687047DC65FF1F9D
:105F8000074B10B5DA68136801331360054B1878B6
:105F9000FF2803D08021C90104F06EFF10BDC04668
:105FA000DC65FF1F8444FF1FF7B50E0002F0B8F850
:105FB000051E1CD00E4B06621F78002F00D10778FB
:105FC000AB791020019304F0E7FF041E0FD0D0231B
:105FD0000380C73B8370019BE91DC3700622043018
:105FE00004F09AFF21003800E66005F065F9F7BD7E
:105FF0008244FF1F014B18787047C046FC65FF1FA5
:10600000054B002805D1054B1A78054B002A00D115
:10601000014B18007047C046EC65FF1FFC65FF1F71
:10602000D665FF1F014B58687047C046DC65FF1FEF
:10603000024B1868431E9841C0B270470066FF1FAC
:10604000421E03000120152A03D9FF3B5A42534147
:10605000D8B27047F0B51C0000230E0085B0039045
:1060600002920B70029A934201D3002019E0E55C82
:106070005A1CD2B2002DF8D0029851198142F4DC9A
:106080000233DFB2A35C18000193FFF7D9FF0028A9
:1060900007D0013D019A0399EBB233708A4202D1D5
:1060A000E01905B0F0BDDB19DBB2DBE710B50C0081
:1060B00002F08EF803001220002B03D02100588834
:1060C00005F042F810BD000070B50E4D8400635914
:1060D000002B15D0186A002801D004F085FF2B5939
:1060E000586A002801D004F07FFF2B59986A0028D5
:1060F00001D004F079FF285904F076FF00232B51DA
:1061000070BDC0460C66FF1F1C4B70B504000E002E
:10611000150099420AD11A4B1B68002B01D112209D
:1061200070BD1B68002BFAD09847F9E7154B9942D0
:1061300015D1134B1B68002B0AD01B68002B07D00E
:106140009847002804D1104B1C70104B1D70E7E7D6
:1061500029002000FFF7AAFF0028E1D1F3E708009B
:1061600001F0DEFF0028DAD003780320A342D7D164
:106170002900300004F0E8FFD2E7C046FEFF00002F
:106180000866FF1FFFFF00000566FF1F0466FF1F74
:10619000F7B50400808801F0C3FF0025A84203D0B2
:1061A0000578A08801F0F8FF1C4E3378002B1FD033
:1061B000AB421DD11A4B28001978FFF777FF002852
:1061C00018D000233370A3790820A778A6880193FC
:1061D00004F0E2FE011E0DD0D0230370CA3B837091
:1061E000019B477086808371280005F065F801E007
:1061F000002DE8D1A0880B4B8200D358002B01D092
:10620000FFF762FF1721A088FFF768FDA08801F063
:1062100017FDA08801F0EEFDF7BDC0460566FF1F23
:106220000466FF1F0C66FF1FF0B587B01D000CABA6
:106230001B88070001930DAB1B88142002930EAB43
:106240001B88160003930FAB1B880091049310ABBF
:106250001B88059304F0A0FE041E1AD0D0230370FF
:10626000CB3B47708370C670062229000430002D96
:1062700011D004F051FE019B21006381029B009824
:10628000A381039BE381049B2382059BA37405F0F8
:1062900013F807B0F0BD04F087FEECE7F7B5009304
:1062A00008AB1B8807000C200D001600019304F0BA
:1062B00073FE041E13D0280001F032FF00280FD017
:1062C0000078D0232370C93BA370009B2100238159
:1062D000019B6770A580E680638104F0EDFFF7BD48
:1062E000014B1878EDE7C0468444FF1F13B5040046
:1062F00064890389C2888188C0780094FFF7CEFF43
:1063000013BD000010B5044C2068002803D004F031
:106310006BFE0023236010BD1066FF1FA122F0B5A5
:10632000818892004A43384B384F1B6804009B1801
:106330009D2292009B18827989B01A603B68002BDD
:106340005FD01D78324B1B68002B04D05B68002B9C
:1063500001D000209847260008363100E079FFF789
:10636000B7FD237DE0710200E0780493638A290081
:106370000393238A0293E3890193A3880093330054
:10638000FFF752FFE378002B0BD1E289A379A188B4
:1063900002920196E27928000092012201F0CAFEE1
:1063A000E0703B68002B20D0FFF7ACFF194D287838
:1063B00000281AD0184B1978FFF778FE002814D05F
:1063C0002B78E67808200793A78804F0E5FD011EE6
:1063D00009D0D0230370CA3B4670837087808671D2
:1063E000079804F069FF00232B701721A088FFF79E
:1063F00075FCA08801F024FCA08801F0FBFC09B02A
:10640000F0BD064B9DE7C0463409FF1F1066FF1F15
:106410002466FF1F0566FF1F0466FF1F8444FF1FDD
:10642000F8B5070008000E0001F07AFE041E18D02F
:106430002620FFF78DFC051E00D12578062004F0EC
:10644000ABFD041E0DD00021062204F0ADFDD023CB
:106450002370C23B21006770A370A680E8B204F0ED
:106460002BFFF8BDF0B585B001930AAB1B78070090
:1064700002930BAB1B7808000D000092039301F010
:106480004FFE061E22D0102004F086FD041E1DD0F3
:106490001022002104F088FD2620FFF759FC002877
:1064A00000D13078D0232370C13BA370009B210022
:1064B0002372019B67706372029BA580A372039B8A
:1064C000C0B2E3720C9BE36004F0F6FE05B0F0BDD1
:1064D000F7B50D00019001F023FE071E20D00E201D
:1064E00004F05AFD041E1BD02620FFF731FC061EC7
:1064F00000D13E78D0232380C53B0622A370F91D2E
:10650000E01C04F009FD019B2A0063810123DD40AA
:106510001A401D40210022736573F0B204F0CCFED6
:10652000F7BD0000F0B585B0029010000D00170017
:106530000A9E039301F0F4FD041E31D0029B002B50
:106540002ED1039B02795B0724D512231343042227
:10655000002E08D10B99002905D10C99002902D1F0
:106560000D9900291AD01A430D9B2271002B00D0DF
:10657000C9E0002E00D1CFE0002D00D0CCE0606A51
:10658000002801D004F030FD1C21300004F0B4FEDE
:10659000606205E002239A430E33D7E793432371E9
:1065A000654BBA00D458002C00D1AAE0002E10D0C0
:1065B000236A002B03D11C2004F086FD20625E4B71
:1065C000BA00D358186A002803D01C22310004F006
:1065D000A3FC0C9B002B12D0574CBB001D596B6ABF
:1065E000002B03D1162004F06FFD6862BB00E35856
:1065F000586A002803D016220C9904F08DFC0D9BDC
:10660000002B11D04C4DBC006659B36A002B03D14E
:10661000142004F059FDB0622B59986A002803D069
:1066200014220D9904F078FC380001F079FD051E64
:1066300067D0414BBA00D358002B62D01A6A34207D
:10664000002A00D11C389A6A002A01D0143080B286
:106650000B9A002A01D01C3080B25B6A002B01D05B
:10666000163080B204F098FC041E4AD01822002193
:1066700004F09AFC2620FFF76BFB0190002801D163
:106680002B780193D0232370029B200063700A2390
:10669000294EA370039BBD00A371AB59A780196A53
:1066A0001830002905D01C22A06004F035FC200021
:1066B00034307359996A002907D003001422143327
:1066C000E060029304F028FC02980B9B002B08D09A
:1066D00003001C221C330B992061029304F01CFC64
:1066E00002987359596A002903D01622606104F098
:1066F00013FC6B462100187904F0DEFD3800FFF72B
:10670000E3FC05B0F0BD10220D9B0D991B69A0188C
:10671000236204F001FC2CE70B9B002B00D13FE728
:10672000012D00D03CE7606A002801D004F05CFC39
:106730001C210B982AE7C0460C66FF1F10B5044CBD
:106740002068002803D004F04FFC0023236010BD14
:106750000066FF1F0B4B07B51A68002A01D1002005
:106760000EBD6946531C012012780731FFF772FCF9
:106770000028F4D002780123100018401A42EED00D
:10678000EEE7C0461C66FF1FF0B51F4F01203B68B7
:1067900087B0002B25D09B78059300F0B3FB002831
:1067A00021D00A20FFF7D4FA04000B20FFF7D0FA1B
:1067B000164B05001E78731E9E413B68F6B2191DEC
:1067C000D878FFF757FB3B682900DA7A0433039245
:1067D0009A7901930292009033002000059A04F008
:1067E0008BFC07B0F0BDFFF7B5FF002805D00620F1
:1067F000FFF7AEFA04000720D8E70820FFF7A8FA51
:1068000004000920D2E7C0460066FF1FFC65FF1F99
:1068100070B50A4E040033780D00FF2B0DD0042014
:1068200004F0BAFB011E08D0D0230370CE3B4570A4
:106830008370C470307804F03FFD70BD9444FF1F36
:1068400070B5040006200D0004F0A6FB011E0AD05E
:10685000D0230370CD3B8370054B44701B6885804B
:10686000187804F029FD002C01D0FFF767FF70BDF8
:106870000066FF1FF8B5264F06003B680D00112487
:10688000002B05D10522234B1B78134202D1122481
:106890002000F8BD204A10241268002AF8D012788F
:1068A000002AF5D0DB0719D52B789A1E012A1AD8B1
:1068B0000C2004F009FC132438600028E8D00023E1
:1068C0000A22437029000670023004F025FBFFF70E
:1068D0005BFF041E0AD0FFF731FFD9E700F012FB7F
:1068E0000028E1D1E4E7002BE2D0D0E70B4B1B7886
:1068F000032BCDD11D20FFF72BFA094B1880002860
:10690000C6D0084B04211878074A04F085FBBFE77E
:106910000066FF1FFD65FF1F1C66FF1FFC65FF1F54
:10692000FA65FF1F2866FF1F60EA0000F7B50193B4
:10693000194B14001A78052306000F0012201A4282
:1069400021D0012920D1154B1D68002D1BD002201C
:106950001F2C18D8002C02D0019B002B13D0104BF9
:106960001F221E706E1C0021300004F01DFB0199D7
:106970002200300004F0D0FA310020002C70002FEB
:1069800006D004F029FCFEBD064B12201D68DCE792
:1069900004F04AFAF7E7C046FD65FF1F1C66FF1FBB
:1069A0009444FF1F1866FF1FF8B50F4E122433687A
:1069B000002B17D01B780F3C834213D100250B4FBF
:1069C0000221387804F0F0FC094B042138781D804E
:1069D00004F0EAFC074B28001D8033685C7004F06B
:1069E00093FB04002000F8BD0066FF1F2866FF1F10
:1069F0001466FF1FFA65FF1F70B5012823D11B4CD9
:106A00002388002B03D01A4A1578002D07D0194B84
:106A10001B68002B02D01878FFF7C6FF70BD3B2B18
:106A200002D93C3B2380F9E7134E0221307804F071
:106A3000BBFCFA222388920002215A43307804F0EA
:106A400033FC2580EAE70B4B1B68002BE6D00B4B91
:106A50001B785B07E2D5084B0221187804F0A4FCF0
:106A60000022024B1A80FFF769FED7E71466FF1F6A
:106A7000F865FF1F0066FF1F2866FF1FFD65FF1FEB
:106A8000F8B51E4D2868002803D004F0ADFA0023A5
:106A90002B601B4E3068002803D004F0A5FA0023B9
:106AA0003360184F05243B7818002040234221D042
:106AB000154800F02BFA3B78234213D0202004F035
:106AC00003FB2860002813D02022002104F06CFA78
:106AD000202004F0F9FA041E306005D020220021A5
:106AE00004F062FA002004E0286804F07DFA2C60CB
:106AF0001320F8BD00F00AFAF4E7C0461C66FF1F39
:106B00001866FF1FFD65FF1F8844FF1F10B50A4C64
:106B100023681A1E0ED0002808D10130587004F0E6
:106B2000F3FA002805D02368002B02D00021FFF7DC
:106B300087FE0122100010BD0066FF1FF7B5274E2B
:106B4000050033680191181E21D05C78244F012C78
:106B500030D1FFF7FFFD002825D02000FFF7F8F81F
:106B60000400412814D91F4B022118781E4A04F052
:106B700053FA1E4B3C3C1C80022233685A703B780F
:106B8000002B14D128000199FFF75AFE0120FEBD09
:106B9000FA2292004243002AEED0124B02211878CA
:106BA00004F082FBE8E7FFF7D3F80200F3E70023E5
:106BB0003B70EBE73B78002BE8D1032004F0ECF9C5
:106BC000011E08D0D0230370CC3B4570837033681E
:106BD000187804F071FBFFF7B1FDD7E70066FF1FDF
:106BE000F865FF1F2866FF1F60EA00001466FF1F9C
:106BF00010B51749838802008B4220D011D815495F
:106C00008B4217D0144900205B1899B2012907D88C
:106C1000926811785A425341D8B2FFF7F9FD01202A
:106C200010BD0E4A00209B1807229BB29A42404199
:106C3000C0B2F5E783681878FFF768FFF0E783686C
:106C400099785A78090218781143FFF777FFE7E738
:106C50000A20000006200000F8DFFFFFAFDFFFFF83
:106C6000014B18707047C0469544FF1F10B5064C85
:106C7000207001F031FA207804F0AEFB0521207875
:106C800000F052FD10BDC0462866FF1F0BB273B561
:106C90000D00002B00DBC4E0884B187804F014F9D9
:106CA000041E0ED00378912B0FD0A22B00D1A1E0AF
:106CB000834B1878FF2852D0210004F0FDFA0028F9
:106CC0004DD180200002684076BD43780F2B76D0EE
:106CD00013D8052B70D00E2BEAD18088794B9842BF
:106CE0002BD8794B98421BD8784B9842E0D1A368B7
:106CF0001878591CFFF774F838E03E2BD8D1837808
:106D0000032B74D06CD8012B6ED0022BD0D1704BDA
:106D10001B68002B23D05B68002B20D098471EE017
:106D20006C4BC0180C28C3D804F096FA1DC2C215CB
:106D30000BC20B0B0B3223C23C00674BC018072859
:106D4000B6D8664B1B68002B09D01B68002B06D0F9
:106D5000200098470AE0A3681878FFF7C7F82000DA
:106D600004F08AFAADE7A068FFF762F800289FD028
:106D7000F5E7A3681B78002BF1D0554B1B68002B5F
:106D8000EDD01B68002BEAD0210055489847EDE76D
:106D90004F4B1B68002BE2D01B68002BDFD021007B
:106DA0005048F3E7504B1B68002BD8D05B68002B92
:106DB000D5D021004348E9E7FFF7EAF9CFE780881B
:106DC0004A4B984203D04A4B984200D070E7464B5A
:106DD0001B68002BC3D05B68002BC0D02100D5E717
:106DE000153B012BBBD963E7FFF798FAB7E7FFF72D
:106DF0007DFAB4E73F4B1B78042B07D100236A468A
:106E000013800179408800F0B5FCA8E7364B1B6879
:106E1000002BA4D05B68002BA1D001003648984716
:106E20009DE7012421420AD0294B1B68002B04D086
:106E30005B68002B01D000209847012043E78B07B7
:106E40000AD5264B1B68002B04D05B68002B01D0B1
:106E500020009847022036E70421280008400D4210
:106E600000D131E7254E3388002B21D0013B9BB266
:106E70003380002B1AD1FFF7DBF800280AD0204B13
:106E80001C70164B1B68002B04D05B68002B01D0D4
:106E900020009847FFF7C6F8694601F0F1FC684604
:106EA000FEF7FEFF1D20FEF753FF308004200AE7A7
:106EB000024B187804F078FAF8E7C0462866FF1FFE
:106EC0009544FF1F0E200000012000000910000063
:106ED0002066FF1FFEDFFFFFAFDFFFFF2466FF1FFF
:106EE0000C2000000B2000000866FF1F0D20000092
:106EF00013200000FD65FF1FFFFF0000FA65FF1F64
:106F0000F865FF1F10B501F08BF910BD014B18603B
:106F10007047C0462466FF1F0B880020162B01D83F
:106F200017230420014A13807047C046D265FF1F13
:106F300000207047074A03001188814207D09188DA
:106F40000020994202D101308000101870470020C3
:106F5000FAE7C0463066FF1FF0B58F7806000D00D7
:106F6000C7B01E2F15D1FFF7E5FF051E03D1002482
:106F7000200047B0F0BD00223B003100C0780092F5
:106F800000F0A2FB0400A81C00F0C3FBFF23EB7081
:106F9000EEE7264B062403931B78FF2BE8D0182F2F
:106FA000E6D87B08224A013BDB0002929A589446BD
:106FB000002ADDD0029AD3185B68002BD8D008785D
:106FC000002802D14B78012B02D10624122FCFD1F9
:106FD00007AFAB88697800976446AA68A047041E8B
:106FE000C6D1AB78029A5B08013BDB00D3183900AD
:106FF00030005B689847041E0BD1AB78042BB6D0E9
:10700000039A310010782200009700F05DFB040025
:10701000AEE76A78002AABD1AA7805A93B88087147
:1070200030000A704B80FEF747FBA0E79844FF1F33
:10703000BCB600111D4B37B5050098420BD0002996
:107040000AD1FFF777FF002805D11948FFF772FF33
:10705000002800D0058037BD01291AD1FFF76AFF4B
:10706000041EF8D001235B420380A378FF2BF2D0EB
:10707000FE2B07D00023E0781422009329001E3352
:1070800000F022FBA01C00F044FB01235B42638064
:10709000E1E70229DFD1013901F0AEF80028DAD1A9
:1070A0002800FFF747FF041EDFD1D4E7FEFF0000F2
:1070B000FFFF0000022210B5074B52421A8007481A
:1070C00001325A809A80DA8000F06EFA044801F0AA
:1070D00015F8002010BDC0463066FF1F596F001123
:1070E000357000110388F7B50400002B02D102258A
:1070F0002800FEBD42680221137825485268FEF739
:10710000A5FD00282ED0234F01253A88002AEFD074
:10711000802321885B0201259B1A9942E8DC0C2020
:1071200003F0D2FF061E31D03B8822889C46002304
:107130001800019561469DB2491989B2AA421BD82F
:10714000002801D062443A8000233000082208C0A1
:10715000210003F0E1FE104A1368002B13D1002533
:107160001660C5E76268022113780C485268FEF782
:107170006DFD0028C7D1BAE760681D014019418143
:1071800001330198D6E71A001B68E6E71325AFE73D
:107190002AB700119644FF1F2C66FF1F28B7001165
:1071A000014B18707047C0469844FF1F14230A0013
:1071B00010B51A40194204D00122102101F038F80C
:1071C00010BD4B06F9D4012088434000F8E710B504
:1071D00014008B0604D50122102101F029F810BDFE
:1071E00008230A001A40194202D14BB2002B0FDAD1
:1071F000102101F01DF8002808D02300F9331B7876
:10720000002BECD0F8342378012BE8D10020E6E7FE
:1072100003208907FAD4E2E7F0B51F00184B85B0C8
:107220001C68019002910392002C27D1200005B028
:10723000F0BDA5683301ED186B89019A934211D313
:10724000029A93420ED8002F04D10A9B002B10D132
:107250002C00EBE73B002978039A6868FEF7F6FC00
:107260000028F2D10136B6B2A388B342E1D824682F
:10727000DAE7A3680A9A5B891380E9E70026F3E757
:107280002C66FF1F37B50C000A88498801239142FC
:1072900017D3002A15D0651D23792A0002210A4838
:1072A000FEF7D4FC102300280BD0237961882088B6
:1072B00000242A000094FFF7AFFF0A23A04200D069
:1072C000230018003EBDC0462AB7001113B50A00BE
:1072D00008884988012388420BD8002809D0002457
:1072E000137905320094FFF797FF0A23A04200D0DC
:1072F0002300180016BD13B50A0008884988012329
:1073000088420BD8002809D0002413790532009454
:10731000FFF782FF0A23A04200D02300180016BD09
:10732000F0B58BB003904A8808880E000123824292
:1073300055D3002853D00023012704AC237000222A
:10734000718813000092FFF767FF051E3ED020787A
:10735000002835D12B78022B18D167706A898300F9
:107360000130E31880005A8069680222201803F077
:10737000D3FD23780133DBB22370042B19D93B00F2
:107380006889013080B2002BD9D01FE002236370DE
:10739000122358436A89231804305A8069681022DE
:1073A000201803F0B9FD23780133DBB22370002BE2
:1073B000E5D10C4A6B899B185A425341DBB2DFE797
:1073C0006378012BE4D12B78022BC7D022780A23D3
:1073D000002A04D021000398FEF798F90023180032
:1073E0000BB0F0BD0100FFFF0F4BF0B504001868B3
:1073F000002816D083685D89A54207D88288AE1818
:10740000B44203DA12019A18934201D10068EFE7FF
:107410001E005F891036A74204D1002900D00D80DC
:107420001800F0BD3300EFE72C66FF1F70B50500B4
:107430000C0008880021FFF7D7FF03000120002B74
:1074400004D022002800197AFFF7C1FE70BDF7B5FD
:107450000C00002501902300F6331B78AB4201D8C5
:1074600000200AE06B00E65A00213000E718FFF721
:10747000BBFF002802D126800130FEBD017A0198B1
:10748000FFF794FE002802D03B882380F5E7013502
:10749000EDB2E0E710B5040008880021FFF7A4FF73
:1074A00003000120002B03D02000197AFFF77EFE95
:1074B00010BD0000054B1B68002B01D1180004E033
:1074C0009A6852898242F6D1988870472C66FF1FCD
:1074D000F0B50E27002687B0039302ABFF183E805D
:1074E00005001F4B40891400984207D02B780130CB
:1074F00000976A6880B2FFF78FFE060002212B78A2
:1075000018486A68FEF7A2FB00280FD06C8920009B
:10751000FFF7D0FF002802D0013C0419A4B2039B5E
:10752000002B00D01C80300007B0F0BD02212B786A
:107530000D486A68FEF78AFB0028E7D102212B7804
:107540000A486A68FEF782FB002807D0002EDED0CA
:107550003B88A342DBD17489013CDFE76C89DEE71D
:10756000FFFF00002AB7001128B7001126B700114D
:1075700070B504000D001600FFF7DCFC002803D0F6
:1075800083781720FE2B05D0002E04D1290020007F
:10759000FEF738F970BD01221021200000F048FEEE
:1075A0000028F3D0F6E70000014B18607047C04692
:1075B0003C66FF1F37B56B469D1D0100040002228B
:1075C000280003F069FD2B88B02B0ED12379122BF4
:1075D00009D12300FF339B78012B06D1012160885C
:1075E00000F0E0F801E01B2BF8D037BD10B5054BDB
:1075F0000421187000F098F8FFF75CFDFEF780FB9F
:1076000010BDC0464066FF1F0020F0B50BB20F0052
:1076100087B0834234DA274B187803F055FC051EF7
:107620002BD00378A02B25D103AE3100FEF7F4F860
:10763000041E0BD1B378DB0724D51F4B06341B681F
:10764000002B03D03100688898470400A868002800
:1076500001D003F019FC002C08D1184A039B1340F9
:10766000174A934206D0B3781B2B03D001216888B8
:1076700000F098F8280003F0FFFD80200002784019
:1076800007B0F0BD0F4B1B68002B10D0310068888D
:107690009847041EDAD07378002BD7D1B27801A9AD
:1076A0000A704B800C716888FEF706F8CEE7062456
:1076B000F1E7C0464066FF1F3866FF1F00FFFF006E
:1076C000000112003C66FF1FF7B5019082204000C8
:1076D0000D0017001E0003F05FFC04001320002CB7
:1076E00012D0B02320002370089BFC2267706580B5
:1076F00026710830002B08D0190003F00DFC210082
:10770000019803F0D9FD0020FEBD089903F04CFC60
:10771000F5E710B5041E06D00078FD2803D803F065
:10772000DBFBFF23237010BD0A1F93B210B50400CA
:107730000220032B05D882400020024BD1529B1817
:107740009C7010BD6066FF1F0B8870B5043B040081
:107750000D000220032B0BD80121200000F04CFD6E
:1077600003001420002B03D02900200000F0DEFBD2
:1077700070BD000007B51300034A00920A00012102
:1077800000F02CFC0EBDC046B179001107B5019286
:1077900003220092024B0A00122100F049FC0EBDA8
:1077A0002F7A001107B56B4601AA11800449D880D1
:1077B00008780633012802D1190003F08DFC07BDBB
:1077C0004166FF1F0C4B10B518700023FF210B4AB8
:1077D0001380138193819380094A538013705172EF
:1077E00093819372D174D3821375517703F024FD82
:1077F00000F0FCF910BDC0467066FF1F6066FF1FF9
:107800004266FF1FF0B58DB06B46002003910C223D
:107810009B5E834200DBB0E05D4B187803F054FBC5
:10782000051E00D1A4E00378902B00D09DE006AFA8
:1078300001004688380000F013FA79680400002936
:1078400000D19CE03B88052B6ED13B89032B1CD9D2
:1078500005AC200000F0A2F86288172A61D83989A7
:10786000131D994231D17968237804310291D907E7
:1078700038D5607800F08EF9071E06D0002303711A
:107880002378012B08D0132B23D0A868002800D11F
:1078900078E003F0F9FA75E06288029909A800F02F
:1078A000A6F80290380000F08BF909AA2378387AFC
:1078B0000192002231000092029A00F012F9380081
:1078C00000F064F9029B002BDFD0300000F080F95B
:1078D000DBE70378032BD8D16288029909A800F06E
:1078E000D6F8DEE7122B13D1029909A800F0B5F8FB
:1078F000021EEAD127498B88002BC6D0887909A9B6
:107900002378019161780091310000F0EAF8BCE73A
:10791000002302AA93833000617809AAFFF72AFFA7
:10792000B3E71D4B0993F6E7042B02D09A1F012AF7
:10793000ABD8184A043B9B00995A0029A5D0D2180D
:10794000907831003A0000F0AEF800289DD13B88D5
:10795000042B03D001213000FFF724FF012C04D1B8
:10796000A868002801D003F08FFA280003F084FCF7
:107970008020039B0002434018000DB0F0BD012899
:1079800000D182E701213000FFF70CFFEDE7C04690
:107990007066FF1F6066FF1F010017000B78037001
:1079A0004B784370CB788A781B021343438070472F
:1079B0000A88030002700A88120A42700A88012AA3
:1079C00006D14A8882704A88120AC2700420704721
:1079D00002208242FBD14A8804309A704A88120AF7
:1079E000DA708A881A718A88120A5A71EFE710B51C
:1079F0000400012082420CD94B780A781B02134301
:107A00002380834206D1CB788A781B02134363809C
:107A1000002010BD022BFBD1CB788A781B021343C8
:107A200063804B790A791B021343A380F0E70B882C
:107A300003700B881B0A43704B8883704B881B0AAA
:107A4000C3708B8803718B881B0A4371CB88837149
:107A5000CB881B0AC3710820704703000120082A45
:107A600014D14A780878120202431A80CA788878BA
:107A7000120202435A804A790879120202439A801C
:107A8000CA798879120202430020DA80704710B563
:107A900004000120022A05D100204B780A781B023D
:107AA0001343238010BDF8B5060010200F00150009
:107AB00003F072FA04000120002C0ED0A0230C2247
:107AC000290023806780201D002D07D003F024FAB1
:107AD0002100300003F0F0FB0020F8BD03F064FA51
:107AE000F6E7F7B51E00009008AB142017001D78CC
:107AF000019103F051FA041E12D0A2230370019BDE
:107B000047704380099B057146710C220830002B99
:107B100007D0190003F000FA2100009803F0CCFB15
:107B2000F7BD099903F040FAF6E737B5041E0FD008
:107B30004388002B0CD00025C1881323007A17221C
:107B400001950095FFF7CDFFFF23658063722570D7
:107B500037BD000010B50C4904004A88002A09D03E
:107B60008B89002B05D00020CB8A0222834201D0D2
:107B700010BD012213000A20434300204032C854A4
:107B8000C81842800472F3E74266FF1F0023438057
:107B900003707047094B00211A0010B55C88002C57
:107BA00006D01C79844203D10A234B43D01810BD60
:107BB00001310A330329F1D10020F8E74266FF1FA3
:107BC00010B50400407A03F087F9FF23637210BDFB
:107BD0007047043010B580B203F016FC002803D0C3
:107BE0000421494203F050FB10BD000070B5002590
:107BF000104CA0682580A581A580A84202D003F082
:107C000043F9A56000250C4C0C4B606D1D802300D2
:107C100058331D70A84202D003F036F9656500257F
:107C20006068002801D003F02FF9013508340A2DCF
:107C3000F6D170BD0867FF1FAC66FF1FFC66FF1F13
:107C400070B5041E09D1054D2880A881A880A868B8
:107C5000002802D003F018F9AC6070BD0867FF1F60
:107C6000F0B54B8885B00193002343600A79050085
:107C70000F00022A00D07BE0CA88032A17D98B683C
:107C80005E7819783602DC78D8790E4399781B7AB9
:107C900024021B020C43034353495BBA0B80331D80
:107CA00093421ED1042C04D0631F022B0ED9012055
:107CB00015E0019A4D4B1201D35A002B06D00198C2
:107CC000FFF7BEFF4A4A1369013313610421B86804
:107CD0002E812C80494203F0D7FA6860002005B05D
:107CE000F0BD434D042C06D0631F022B0FD9EB6867
:107CF0000133EB60DBE7019A3C4B1201D35A002BB6
:107D000005D00198FFF79CFF2B6901332B61374B9E
:107D100030000293019B029A1B01019300230199F9
:107D20008C468B52130063449C8003939E81FFF723
:107D300050FF039B041E986016D00421B868494286
:107D400003F0A2FAFA880100043A200003F0E4F8F4
:107D50000199029AFB888A5A043B9B18029A8B521B
:107D60002B6801332B60A2E7AB690133AB619EE75F
:107D70001E4B0293019B1E01029BF35A002B2DD038
:107D800002998C19A068002828D0012A26D1FA88E7
:107D90009B189BB27352A189994217D39B1AC018A2
:107DA000B96803F0B9F8029BA289F35A934200D054
:107DB0007DE700222B81A3882B80A3686B60029B48
:107DC000F2520B4A53680133536070E7084A9368D4
:107DD000013393600198FFF733FF68E7044A536962
:107DE00001335361F6E7C0467266FF1F0867FF1F45
:107DF0007866FF1F70B5051E15D10B4C0B4B188014
:107E0000230058331870606D002802D003F03CF84E
:107E10006565250050356068002801D003F034F80E
:107E20000834AC42F7D170BDAC66FF1FFC66FF1F83
:107E3000F0B51700A12285B0920001934243394B5F
:107E400006001B680C009B18D933FF331D78FDF723
:107E500051FF0430854204DD3000FDF74BFF043054
:107E6000C5B2BD4207D33A0000213000019B03F0A8
:107E7000E3FA05B0F0BD2900380003F0B5F923009E
:107E8000C6B250331E700393019B2900636538000E
:107E900003F02AF9CBB20293002B02D0039B0136E8
:107EA0001E7000262300503303931B78B34204D87E
:107EB000606D002831D10020DBE7029A2800002AFB
:107EC00004D0013B1000B34200D02800F700E719AE
:107ED000387002F0E9FF786000280ED03A780199F6
:107EE00003F01AF8019A3B780136D3180E4A019331
:107EF000D369F6B20133D361D4E7039B1870606590
:107F0000A74205D1084A1320D36A0133D362B0E7F0
:107F1000606802F0B9FF0834F2E702F0B5FF002311
:107F20006365C8E73409FF1F7866FF1FF7B50D00CA
:107F300007000421686803F0A7F92B890400037087
:107F40002B891B0A43702B8883702B881B0AC370F4
:107F50002E8902250436F6B2FB2E15D81B4B9F4204
:107F600014D10C2003F018F81135011E0CD0902309
:107F700003708E3B0371043B4380154B8460C680C5
:107F8000187803F099F900252800FEBD5C237B4397
:107F9000104AD3180093583301931B78002B0FD14C
:107FA0000300320038000099FFF742FF019B0500F3
:107FB0001B78002BE8D13800009903F005F9E3E7BE
:107FC000054A0725536A01335362DDE7FEFF0000CF
:107FD0007066FF1FAC66FF1F7866FF1FF0B587B0A5
:107FE000009017200F0016000193FFF7F2FD1325F4
:107FF000041E19D00C98031E02D00199201D984729
:10800000030AE370052302AAA07004309081277050
:108010000098667003A993800494FFF787FF051EFC
:1080200002D0200002F030FF280007B0F0BD0000B1
:10803000F0B587B01F000CAB1B78039105930121AD
:108040000DAB06001C78049200F0D6F81425002829
:1080500021D02000FFF77EFD0135041E1BD0114901
:10806000059B0A7803700132D2B2131EC68001D17B
:1080700001231A000B7022713000049B03990097B2
:10808000FFF7ACFF051E09D1230021000648074A6F
:10809000093303F091F8280007B0F0BD0023638096
:1080A0002370F8E77466FF1F2B7B0011307500000A
:1080B000F8B505000E00064C064F2368002B02D0D1
:1080C0003100280098470434BC42F6D1F8BDC046C0
:1080D0001867FF1F2C67FF1F0123064A5B4253806E
:1080E000002313715362044A136053609360D3609A
:1080F000136170472C67FF1F1867FF1F02000023E2
:1081000010B506499C000859002801D1625010BDE5
:108110000133052BF6D11320F9E7C0461867FF1F7E
:10812000034A5388181A434258414042104070474E
:108130002C67FF1FF0B585B002930AAB1F780CAB1C
:108140001B88009008000E0001920393FFF7E8FFE0
:1081500005001120002D1BD10E48FFF7E1FF0400A0
:108160001520002C14D006220B99A771E01D02F0F7
:10817000D3FE019B30002371029B29006371009B99
:1081800066802370039B6562E381FFF791FF2800FF
:1081900005B0F0BDFFFF000010B5FFF7C1FF040000
:1081A0000220002C12D060880121FFF781FF606A55
:1081B000002801D002F018FF28220021200002F040
:1081C000F3FE012300205B426380207110BD00009C
:1081D00030B5074A074C5588010013780020A542A6
:1081E00004D05B1A59424B415842104030BDC04642
:1081F0002C67FF1FFFFF0000084A10B501230C0089
:10820000904208D0FFF78CFF031E04D0037923406F
:108210005A1E9341DBB2180010BDC046FEFF00009D
:10822000024B1879431E9841C0B270472C67FF1F5C
:1082300070B504000D001600FFF772FF002804D18E
:108240000D4B9C4200D0143070BD416A037905206B
:10825000002907D012221A40102A02D10520002E30
:10826000F2D10F20DB06EFD5897E0C20A94289418F
:10827000494249420840E7E7FEFF0000030010B50D
:10828000002800D110BD0348034A41889142F9D02B
:108290009847F7E72C67FF1FFFFF0000002330B56A
:1082A000C45CCD5C6C40D4540133102BF8D130BD8C
:1082B0000F23002210B5C45C64002243CA54C25C80
:1082C000D209013BF7D210BD0200010010B52032E7
:1082D000103103F029F810BDF0B58BB003901020D9
:1082E00005931700049102F0EFFE0090102002F0B9
:1082F000EBFE009B13240190002B05D000280CD12D
:108300001324009802F070FE019B002B02D018008D
:1083100002F06AFE20000BB0F0BD102002F0D4FE87
:108320000600102002F0D0FE13240500002E00D11C
:10833000AEE0002819D01022002102F035FE3200F4
:108340002900039802F0F0FF041E0ED133787F2B32
:1083500051D830000099FFF7ABFF009B1B787F2BB3
:1083600053D801990098FFF7A3FF300002F03CFEBC
:10837000002D02D0280002F037FE002CC1D11020C1
:1083800002F0A2FE0600102002F09EFE0290002ED7
:108390007CD0002878D03A000F322300012512113A
:1083A00005D00F333B4015B25A4253411BB26A1EEF
:1083B0001201002B33D0049BD2B298180099029A74
:1083C000FFF76CFF013D10220021300002F0ECFDB0
:1083D000ADB2049F2D017D19AF4242D0002C33D0A5
:1083E000300002F001FE029B002B00D189E718004B
:1083F00002F0FAFD85E729003000FFF759FF280059
:108400002549009AFFF74AFFA7E729000098FFF7E0
:108410004FFF28002049019AFFF740FFA5E70F21F1
:108420000F4004998A18D9B28F4208D9D15C06A8A6
:1084300019540133102BF6D1029A0199C0E7791A29
:1084400048424141C901F2E73900300006AAFFF76E
:1084500025FF3200039806A902F066FF10370400DA
:10846000BAE7002CBCD13000029906AAFFF716FF2C
:10847000320006A9039802F057FF082204003100D9
:10848000059802F049FDABE71324A9E71324AAE7F6
:10849000002800D06EE733E730B70011F0B58BB09D
:1084A0000F0016000225009000283FD0002A3DD082
:1084B0000B1DDBB21800029302F006FE1135041EFC
:1084C00034D0FDF757FD05003A000099201D02F059
:1084D000EBFFEBB20393E3702B0CDBB22F0A00939C
:1084E0006370FFB22B0E2370A7700193FDF73CFD64
:1084F0001022010006A802F0D7FF2100029A04AB67
:1085000006A8FFF7E9FE051E0DD1039B0822337074
:10851000009B04A9B370019B7770F370301D02F0CB
:10852000C3FFFDF72DFD200002F05EFD28000BB01B
:10853000F0BDF0B58FB00D00149E0390049205932A
:10854000002A03D1022420000FB0F0BD002EF9D084
:108550000398FFF7E5FD1424071EF4D072783378F2
:1085600012021A43B3781B041343F27812061A431B
:10857000036A0192934201D30133E3D1002D03D06A
:108580003B7901249B07DED50822002106A802F0D2
:108590000BFD059B13240433DBB21800029302F099
:1085A00093FD051ECFD0059A0499043002F07CFF9C
:1085B00004223100280002F077FF39001022103128
:1085C0000AA802F071FF2900029A06AB0AA8FFF779
:1085D00083FE041E0FD1082206A908A802F064FF3A
:1085E0000822311D08A802F00FFD012807D10199CA
:1085F0000398FDF7D9FC280002F0F6FCA3E701245C
:10860000F9E7000070B51C4C05002368181E10D057
:10861000002D14D11A78002A0CD1981C083202F0CF
:108620007BFC02F079FD0135002808D123681D701C
:10863000012070BD0A331800082202F06DFC236887
:10864000002BF5D0122002F0A7FC061E0DD0C1238E
:1086500021680370457002311022023002F05CFC88
:1086600023683100587802F027FE206802F0BCFC35
:1086700000232360DCE7C0465467FF1FF8B5040001
:108680002020FDF765FB0D4EA700BB590500002B10
:108690000DD000280BD0D878FF2809D108492A002E
:1086A0000C55F35907480333611802F085FDF8BDF6
:1086B000290002F069FD0028F0D1F8E77067FF1F7C
:1086C0005867FF1FD598001170B5064D8400635997
:1086D000002B05D0D87802F0FFFBFF226359DA7037
:1086E00070BDC0467067FF1F70B506008CB00C00EF
:1086F000150000213022684602F056FC310010229D
:10870000684602F0D1FE1D2021000322684402F0D9
:10871000CBFE6846FFF7D8FD2D2104000322280078
:10872000694402F0C1FE20000CB070BDF0B5070036
:10873000160097B001931CAB1D7830221EAB009140
:108740000AA800211C7802F02FFC102239000AA888
:1087500002F0AAFE1022002102A802F025FC072246
:10876000310002A802F0A0FE072202AB9818631E97
:108770009C41019902F098FE02AB9C732B005A1E9B
:10878000934102AAD3730021102206A802F00CFC28
:1087900006221D9907A802F087FE1A2002ABC01816
:1087A00006221F9902F080FE102200990EA802F006
:1087B0007BFE102202AB0EA908781C78013A6040BB
:1087C000D2B2087001330131002AF5D10AA8FFF7AF
:1087D0007BFD102212A904000EA802F09DFB1022BE
:1087E00006AB0EA908781D78013A6840D2B208702D
:1087F00001330131002AF5D10AA8FFF765FD0443D2
:1088000010222098E4B212A902F04EFE200017B008
:10881000F0BD70B50E0014008CB001001022684647
:108820001D0002F041FE3100082204A802F03CFEC7
:108830002100082206A802F037FE6846FFF744FD33
:1088400004001022280008A902F02EFE20000CB01F
:1088500070BDF8B506000D0000243719AC4200D3F6
:10886000F8BD02F0D9FC030A3B70631CDBB2013790
:108870009D4203D90234F054E4B2EEE71C00EDE768
:1088800073B506000C000225002819D0002917D066
:10889000032101A8FFF7DDFF6B469A793F231A40B9
:1088A000013313436A463000937101A92200FFF798
:1088B0001BFF051E04D10322E01C01A902F02CFBC2
:1088C000280076BD03785807DA08C00FD200800070
:1088D0009B0710439B0F1843C0B2704707230B4000
:1088E000C908C9000B4303707047000070B504004D
:1088F000FFF7EAFE134DA4006359002B21D0186A3C
:10890000002801D002F070FB2B59986E002801D08E
:1089100002F06AFB2B59D86E002801D002F064FBEC
:108920002B59186F002801D002F05EFB2B59586FAD
:10893000002801D002F058FB285902F055FB002313
:108940002B5170BD7067FF1F0E4B8000C35870B570
:108950000C00002B0FD09D68002D0CD02B78201D13
:108960000B706B784B70A97CFFF7B8FF2B7E2372DE
:108970006B69E36070BD10220021200002F014FB3F
:10898000F8E7C0467067FF1F014B18607047C0468C
:108990006C67FF1F074A03008000825810B5002A49
:1089A00006D0D088984203D1012901D1FFF79EFF5C
:1089B00010BDC0467067FF1FF0B5264E95B087000A
:1089C0000B93BB590500099112200A92002B31D05C
:1089D000D888FFF7A5FB04001420002C2AD028001B
:1089E00010A9FFF7B1FFBB591E781D6A002E23D0D6
:1089F0000895FDF7FFFA07000020FDF701FB07903F
:108A0000A379E61D069310AD0CA9089800F0E2FAD0
:108A10000EA9280000F0D7FA0B9B0A990493069B35
:108A200009980293079B0396019300970EAB0CAA3B
:108A3000FFF77CFE15B0F0BDFDF7DCFA06903000C4
:108A4000FDF7DEFAE31DA779079310AB0600089344
:108A5000DAE7C0467067FF1F30B50C4C85002A5915
:108A6000030085B00120002A0ED018006946FFF7E8
:108A70006BFF2B591A78D888054B002A00D1054B7B
:108A80006A46072100F0D9FB05B030BD7067FF1FB3
:108A9000C78F0011D58F001130B5094C85002959B9
:108AA00085B010226846253102F036FA2A59112184
:108AB000044BD0886A4600F0C0FB05B030BDC0460C
:108AC0007067FF1F7190001130B5094C850029595E
:108AD00085B010226846353102F01EFA2A5911215C
:108AE000044BD0886A4600F0A8FB05B030BDC046F4
:108AF0007067FF1FAF900011F7B54D4F8600102033
:108B0000F4590D0002F0E0FAF3592062186A1322BA
:108B100000286CD0033A29009C6802F0FDF9F35953
:108B20001A780192002A58D11E6A227D317B944620
:108B300051400122019F114201D167461740217D1A
:108B4000914339432175377B4F40BC46604600272F
:108B5000800701D44F081740012102208F40227D59
:108B600082433A432275377B5740BC466046002714
:108B7000400701D497080F400420227DBF008243A4
:108B80003A432275627D002794466046727B4240DC
:108B90000A4201D167460F400121627D8A433A4370
:108BA0006275777B5740BC4660460027800701D43A
:108BB00057080F400220627D7F008243174367758C
:108BC000767B00227E40760701D4BA080A4004264C
:108BD000617D9200B1430A4362756A78002A08D029
:108BE0006278002A05D005220533DA7700221000CA
:108BF000FEBD04222979114205D1A17C114202D186
:108C00000533033AF1E7019A21782C78002A02D142
:108C10000A002100140018220429E8D8042CE6D800
:108C200005206043034A05331218525CDDE7C04655
:108C30007067FF1F40B7001110B50A001121024BE9
:108C400000F0FBFA10BDC0460B9100110B0030B5CF
:108C500087B001AD2B806B4604001100981D0822DF
:108C600002F05AF92A000B212000024B00F0E5FA2D
:108C700007B030BD3391001110B50A001121024B2D
:108C800000F0DBFA10BDC0468791001113B50B0050
:108C900011006A4613706B4604000622581C02F04D
:108CA0003BF96A4608212000014B00F0C6FA13BDCB
:108CB000A791001110B50A001121024B00F0BDFA76
:108CC00010BDC046F79100117FB505000B4BAA00FF
:108CD000D4580800002C0FD0666F237FE2882178DB
:108CE0000396266F0296E66E0196A46E0094FDF739
:108CF00019FC2800FFF7FAFD7FBDC0467067FF1F13
:108D000010B51721FFF7E0FF10BD000070B50A0095
:108D10000D00064B0221040000F08FFA06002978AE
:108D20002000FFF7D1FF300070BDC046D790001182
:108D300070B586B000236A461370836804001D78FE
:108D4000681E0A2859D801A902F056F906063337D9
:108D50003B3F43474B4F5300180000F042F90623B6
:108D600012284BD000281BD16088FFF7D9F90823BF
:108D7000002813D04279002A47D1264B1A780723BE
:108D800012070BD5244B1A680723002A06D0166851
:108D9000002E03D0290001AAB04703006A461370D1
:108DA0006B461B786088002B2AD1FFF767FC06B062
:108DB00070BD180000F06CF9D4E7180000F087F9D6
:108DC000D0E7180000F093F9CCE7180000F0ADF9F7
:108DD000C8E7180000F0C3F9C4E7180000F0F6F97E
:108DE000C0E7180000F0F6F9BCE7180000F013FA2D
:108DF000B8E7180000F013FAB4E707236A461370C7
:108E000069466088FFF782FFD1E70523012AC5D1B3
:108E1000024BB8E7FD65FF1F6867FF1F6C67FF1F08
:108E2000F8B52C4F8600F35904000D00002B40D0FC
:108E3000DA8882423DD15A78062A33D11A78002A3C
:108E40002ED0012099681A6A097D014206D0157B4F
:108E5000054203D007225A700120F8BD02200142CA
:108E600004D0157B054201D00922F4E70420014219
:108E700004D0127B024201D00B22ECE7164B1B6898
:108E8000002BE9D05B68002BE6D020009847BB5947
:108E900000215B78122BDFD12000FFF715FFDBE705
:108EA0000E4BECE7112A04D1002900D0322529000D
:108EB000F2E7002D08D12000FFF732F9002803D097
:108EC000102302791343037121002800FDF7A8FA4B
:108ED000C2E7C0467067FF1F6867FF1F6C67FF1F10
:108EE00070B50E4E8500AB590400002B13D01B78D3
:108EF000002B11D10A4B1B68002B04D05B68002BA0
:108F000001D02000984773595B78122B03D10021C0
:108F10002000FFF7D9FE70BD024BECE77067FF1F22
:108F20006C67FF1F6867FF1F094B8000C358102044
:108F3000002B0CD01A6A002A09D09B68002B06D09F
:108F4000127A1B7E101C9A4200D9181CC0B27047BE
:108F50007067FF1F70B503000D0014000220002A87
:108F600030D000292ED013700B78081D53704B7829
:108F70009370FFF7A7FCE070012002212B7A237188
:108F80006B7B034063716A7B0A4013430422637165
:108F90006E7B1640334363716E7BF608F6003343F5
:108FA00063712B7B0340A371287B014000200B439E
:108FB000A371297B0A401343A3712A7BD208D200F4
:108FC0001343A37170BD10B50A0001000120FFF723
:108FD000C1FF10BD10B50A0001000220FFF7BAFF63
:108FE00010BD70B506000C000220002E30D0002904
:108FF0002ED07378201D0B70B3784B70F178FFF78B
:109000006DFC01223579257271794B1008001340EF
:10901000934010400343881010408000C908034368
:10902000C9000B436373B1794B10080013409340A0
:1090300010400343881002409200C9081343C9003E
:109040000B4321202373FCF783FE854201D21220BB
:1090500070BD2220257AFCF77BFE8542F7D8237865
:109060001820042BF4D86378012BF1D80020EFE707
:10907000030010B50220002909D0002B07D00322DD
:10908000481C0A7019000D3201F046FF002010BD87
:1090900003000222080010B5002B06D0002904D0DE
:1090A0000E32591C01F038FF0022100010BD0300E1
:1090B00010B50220002909D0002B07D00422481C3B
:1090C0000A7019000C3201F027FF002010BD10B506
:1090D000FFF7DEFF10BD03000220002906D0002BA1
:1090E00004D0052200200A701B784B7070470300E3
:1090F0000220002B08D0002906D05B7800200B70DE
:10910000013B082B00D918307047030010B502202E
:10911000002909D0002B07D00622481C0A7019002C
:109120000A3201F0F9FE002010BD10B5FFF7B0FFC4
:1091300010BD02000B00022010B500290ED0002A3D
:109140000CD007211970118859701188090A99707B
:1091500011180822D81C01F0DFFE002010BD03000A
:109160000A00022010B5002B0CD000290AD09978F3
:109170005878090201431180901CD91C082201F083
:10918000CBFE002010BD030010B50220002909D03D
:10919000002B07D00822481C0A701900921801F011
:1091A000BBFE002010BD02000B00022010B50029FC
:1091B0000BD0002A09D0092119701178181859709C
:1091C000511C062201F0A8FE002010BD10B5FFF7CB
:1091D0005FFF10BD02000B00022010B5002A09D06D
:1091E000002907D05178197011180622581C01F077
:1091F00093FE002010BD030010B50220002909D005
:10920000002B07D00A22481C0A701900063201F010
:1092100083FE002010BD10B5FFF73AFF10BD02001D
:109220000B00022010B5002A06D0002904D0180037
:109230005178FFF753FB002010BDF0B585B0170043
:109240001E006A4606230500080091819380FEF700
:10925000C0FC1324011E02900CD03800B047041E3D
:1092600005D1280001A9FEF76FFA041E02D002986A
:1092700001F00AFE2800FFF701FA200005B0F0BD5A
:10928000F0B504008BB0019115000021102202A856
:1092900001F08AFE334EA700B85900283CD0C3889D
:1092A000A34239D10378002B36D14278062A18D14F
:1092B00002000100553235310C3006ABFFF7A9FA38
:1092C000002829D12000FFF72FFE020006A902A8DE
:1092D00001F022FE200002A901F046FE01200BB0A1
:1092E000F0BD816E002917D00B8A112A28D19D422A
:1092F0000ED101981231093A01F086FE012807D1FA
:10930000BB5920009D6EFFF70FFE29000200DEE72B
:1093100032212000FFF7D8FC2000FEF701FF061ED7
:109320001BD0416A002918D00B8AAB4215D1082204
:109330000198123101F068FE01280ED1716A0AE02D
:109340009D42E9D108220198123101F05DFE012809
:10935000E2D1BB59996E8A7EB9E7200001F084FE04
:10936000BCE7C0467067FF1FF0B56B4D87007E59A4
:1093700085B0337802900393002B00D087E0B36868
:10938000346A01937078062817D101221B7D13429D
:1093900002D0217B114218D10222134202D0217B3C
:1093A000114251D10422134203D0237B134200D037
:1093B0008BE0019B5A7DEB5991E007380428F8D8DF
:1093C00001F01AFE032E42678300B36E002B03D117
:1093D0001C2001F079FEB066EB599C6E002C1CD06D
:1093E00010220021200001F0DFFD0298FFF79CFD14
:1093F00001002000FFF72DFA01F00EFF208220006F
:1094000008211230FFF725FA0298FFF78DFDA076AC
:10941000EB592100D888FFF70FFC0822EB591CE01C
:10942000B36E002B05D01A00198AF0881232FFF7AC
:109430000DFC0222019B197DEB5911423DD0207B8E
:1094400010423AD0073208E0F488FCF7EBFD010047
:109450002000FFF711FC0A22EB595A70029B9C0076
:109460002A595378073B042B11D8D088FEF758FEB1
:1094700000284ED0C3895A08D2182849029B029866
:10948000CB542B5941180433254801F095FE05B003
:10949000F0BDFCF7AFFD03000120834201D10020A5
:1094A0000393EB59DE88FCF7ABFD03990200300013
:1094B000FFF7ECFB019AEB59117D042211420CD00D
:1094C000217B114209D00B22C7E7F688FCF74CFD3F
:1094D00001003000FFF7EEFB6BE7019A527D01219E
:1094E0000A4204D0607B084201D00C22B5E7022179
:1094F0000A4204D0607B084201D00E22ADE704216D
:109500000A4204D0627B0A4201D01022A5E712224F
:10951000A3E7FA225200B0E77067FF1F7467FF1FCE
:10952000DF98001110B5064B1A780423100018407C
:109530001A4200D00348FFF727FA002010BDC046AA
:10954000FD65FF1F9C44FF1F70B50400FFF7D4FAB0
:10955000051E43D12000FFF77FFA234EA400A05937
:109560008268937CDB0708D50321036A1B790B40D3
:10957000012B02D1017F0B430377431DD97F8B1E43
:10958000022B0DD8022900D00121C088FCF7A0FFD2
:10959000042133591A7F59700A431A77280070BD85
:1095A00001290CD102231022437000210C3001F05C
:1095B000FBFC305910213530FFF74BF9EEE7052958
:1095C000ECD10223D118437010220C3001F0A4FC1E
:1095D00004233259117F0B431377EAE70825182833
:1095E000DCD1053DDAE7C0467067FF1FF0B58BB0F0
:1095F000059143887E4F9E00F45915000493002C7A
:1096000015D1012902D000200BB0F0BD101D5778F4
:109610001678FFF757F9EB68320002932B7A04991A
:10962000019300903B002000FCF71CFFEBE7E38870
:10963000049A934201D00820E6E72378012B00D159
:10964000D4E0059B581E092800D9CFE001F0D4FCD6
:1096500005CE0A29CC506C859AB229000498FFF7F0
:1096600073FFD1E7200029001022453001F054FC9F
:10967000B9594B78042B02D1013B4B70C3E70B0067
:109680000A00253335320C310498FFF795F9049818
:10969000FFF702FA0522431E9841BB59C0005A70D9
:1096A000B2E7200029001022553001F035FC049B60
:1096B0004F4C9D00295904980A0006AB55320C31D5
:1096C000FFF77AF929591022453106A801F09CFCD0
:1096D000012808D10498FFF7F7F90590002804D174
:1096E00006222B595A7005988EE708230593FAE74E
:1096F00063780C2B7AD1E36E002B03D11C2001F090
:10970000E3FCE066BB59D86E00286FD01022290018
:1097100001F002FCBB590498DC6EFFF705FC0D223A
:10972000A076BB595A706EE7E06E00285ED0637871
:109730000D2B5BD12B8808220382A91C123001F06B
:10974000EBFBBB599A68517D0222114226D0186A60
:10975000407B104222D00C32E4E763780E2B45D1D7
:10976000236F002B03D1162001F0AEFC2067BB59FC
:10977000186F002803D01022290001F0CDFB0F2222
:10978000BB59CFE763780F2B30D1206F0622691CBD
:10979000103001F0C1FBBB599A68517D042211427F
:1097A00003D0196A497B1142D5D100210498FFF7F3
:1097B0008BFA28E7636F002B0DD0BB59586F002838
:1097C000F3D01022290001F0A7FB0122BB5952421D
:1097D0005B6F1A61E9E7142001F076FCBB59606702
:1097E0005B6F002BE9D126E72978DFE707200BE73D
:1097F0007067FF1F10B5064C207001F025FB062195
:109800002078FDF791FF0348FEF778FC10BDC046B5
:109810008367FF1F9589001100200BB270B50D0002
:10982000834216DA264B187801F04EFB041E0DD049
:109830000378922B0ED0A02B37D0224B1878FF281C
:109840003AD0210001F038FD002835D180200002F7
:10985000684070BD43780E2B0BD03E2BEDD1837842
:10986000052B12D0082BE8D181798088FFF7D8FA30
:1098700008E0154B82889A42DFD183681878591C1A
:10988000FEF7C0FE002817D1D7E7104B1B785B0707
:1098900012D50F4B1B68002B0ED09B68002B0BD0F2
:1098A000C289811D80889847ECE7FFF741FAA068DC
:1098B000002801D001F0E8FA200001F0DDFCC5E746
:1098C0008367FF1F9544FF1F18200000FD65FF1FE1
:1098D0006C67FF1F10B50078FFF712FA10BD10B5C6
:1098E0000078FFF7FDFA10BD0C234343084A10B57A
:1098F0009B185A68002A03D0012901D1904710BD56
:109900009B68002BFBD00029F9D19847F7E7C046A8
:10991000A067FF1F10B5162813D801238340094AFA
:10992000946B1C439463506B98435063D46B20003A
:109930009843012901D120001843D063116B0B43D8
:10994000136310BD00800040F0B500240127154BC3
:1099500085B0DA6B144E03921A6C0192DA64019BA3
:10996000E3403B4217D0039DE5403D400295E5B200
:1099700002992800FFF7B8FF316A736A002908D0FE
:109980003900002B01D0029979402800FFF7C2FF6F
:1099900001E0002BF9D101340C36172CDFD105B0D2
:1099A000F0BDC046008000408467FF1F10B5012451
:1099B00002002000162A08D8054B5968D1402142E0
:1099C00004D01868D0400123184010BD186DF9E785
:1099D00000800040162807D80122064B824000294B
:1099E00003D0D9680A43DA607047D9689143D960D7
:1099F000FAE7C0460038004030B5162818D80324CE
:109A000044430F4BE25C1B199C785D7801232D1BAE
:109A10000135AB40013BA340A140DB430C001228C1
:109A200007D8084992005218116819402143116063
:109A300030BD054A11680B4023431360F8E7C04668
:109A400087B7001108F0004014F00040C21F70B545
:109A5000D4B20623092C0BD80125084C95400029C7
:109A600008D00021FFF7C8FF23682B4323600023A1
:109A7000180070BD2368AB43F8E7C04600380040CB
:109A8000F0B5162826D8214B1B185B78022B21D164
:109A9000032444431E4A1F4EA35C121994780122EA
:109AA00015008540B76B013CE4B23D43A240B5636D
:109AB000194C122815D89B0000290CD117495B18A6
:109AC00099680A439A600123205C154A8340116813
:109AD0000B431360F0BD11495B189968914399607D
:109AE000F1E70E4B00290DD159690A435A61225CF6
:109AF0001328E8D00123203A93400A490868034319
:109B00000B60E7E7596991435961F0E78467FF1FEC
:109B100087B7001100800040CCB7001100F0004072
:109B2000A0F00040A4F00040F8B500241B4E1C4DEE
:109B30001C4B1B5D012B1FD1184A9269E2401A424F
:109B40000BD00122AA5693402200143AD2B2022A24
:109B500009D815494A6913434B6101340C36023563
:109B6000172CE5D1F8BD0022AA560F4992005218D1
:109B700091680B439360F0E7022BEED1E7B2380017
:109B8000FFF714FF01235840C1B23800FFF778FFF8
:109B90003800FFF70BFF7077DFE7C0468467FF1FD1
:109BA00059B700118567FF1F00F0004001220238FD
:109BB0008240054B002903D059690A435A61704716
:109BC000596991435961FAE70038004070B50400C3
:109BD0000D000520162C1AD800212000FFF7FAFEF0
:109BE000A31E012B03D801212000FFF7DFFF002176
:109BF0002000FFF72BFF01220A49A2400A4B4868C8
:109C0000012D05D102431B194A605D70002070BD13
:109C10009043486002211C196170996991439961D0
:109C2000F4E7C046008000408467FF1F10B5162887
:109C30000AD80122074B8240002906D019680A433E
:109C40001A600121FFF7C2FF10BD19689143196026
:109C5000F7E7C0460080004070B505000520162DCE
:109C600017D80C2300246B430A4A21009B181C7050
:109C7000094B28005B195C70FFF7A8FF0123AB407C
:109C8000200006490A681A430A6005490A689A438F
:109C90000A6070BDA067FF1F8467FF1F348000400B
:109CA0003080004070B504000E00FF2813D003255B
:109CB0000540FFF7D1FF084AA3089B009B183F22ED
:109CC000ED00AA40AE40196820009143314319606D
:109CD0000121FFF77FFE70BD18380040F8B5050080
:109CE0000520162D25D80C246C43124BE41863680C
:109CF000002B03D1A3680D30002B1AD002220127BC
:109D00000D4B00215B195A7028002770FFF75EFF8A
:109D100063681E1E08D0A3683E00002B04D02800F4
:109D2000FFF744FE4640F6B228003100FFF7F2FD8F
:109D30000020F8BDA067FF1F8467FF1FF7B5C42090
:109D4000FF222B4B80001958002491437F3A0A438D
:109D50001A508022274F5202274E1A60274B1D5D52
:109D6000002D21D0A31E012B03D80121E0B2FFF763
:109D70001DFF012D18D11F4B9B69E3402B4213D0CF
:109D8000E3B218000193FFF711FE01000198FFF7FD
:109D90004DFFE3B2143B022B1DD801217156184A26
:109DA0008D405369AB4353613B7F002B0DD0E5B22F
:109DB0002800FFF793FF2800FFF7F8FD7B7F0100E5
:109DC000834202D02800FFF78FFD01340C370236A2
:109DD000172CC3D1F7BD012100237156F3568D40D6
:109DE000074A9B009B189A68AA439A60DCE7C04622
:109DF00000E100E08467FF1F59B700118567FF1F6E
:109E000000F0004010B504000520162C0CD80121EC
:109E10002000FFF7DBFE0123044A002011194B70DC
:109E2000A34091690B43936110BDC0468467FF1F37
:109E300070B50E0015000400FFF70EFF0C236343FE
:109E4000094A20009B189D605E60FFF747FFF021E4
:109E5000064B074A8900051E5A5002D02000FFF722
:109E6000FBFE280070BDC046A067FF1F0000FF1F5B
:109E70004999001170B5134D07202C78002C1FD183
:109E8000982221005200280001F076F90123C42015
:109E9000FF222B700C4B80001C635C630B4B1C601F
:109EA0005C600B4B195891437F3A0A431A50802249
:109EB00052021A600D20074A074901F0ADFA20004E
:109EC00070BDC0468467FF1F00800040A0F00040C6
:109ED00000E100E03D9D0011299B0011030010B539
:109EE0000620072B09D8054A137001F065FAD7211F
:109EF0000020034B034A89005A5010BDC444FF1F81
:109F00000000FF1F151BFF1F70B51D0002240C2948
:109F100010D8094ACA40D2070CD5FBF725FF041E0A
:109F200008D1059A04992800FBF73AFFFCF7A8FD31
:109F3000FFF7F8FA200070BD1210000030B50D7860
:109F400002232C009C43184201D02B431C000825FF
:109F50002300AB43284201D02B00234320241D00C3
:109F6000A543204201D01C4325002A230D7018422E
:109F700004D011781E3B0B43137030BD0028FCD178
:109F80000C2113788B43F7E7F8B51D0006AB1B884F
:109F9000140007AA0E000B201778002B27D10A788F
:109FA000022A49D14A68507811780002244A0843AD
:109FB0008018042840D801F01FF803121D1B23004D
:109FC000F06801F049FA021CC0B2B84200D93A1C4C
:109FD000D2B22000F1682A8000F09EFF06E0022243
:109FE000F3681B882A8023701B0A63700020F8BD69
:109FF0000622EEE701232B80F3681B782370F5E738
:10A00000F368002B16D008222A801A8822701A883A
:10A01000120A62705A88A2705A88120AE2709A88EC
:10A0200022719A88120A6271DA88A271DB881B0A8F
:10A03000E371DBE72B80D9E701202B80D7E7C0460F
:10A0400000D6FFFFF7B516000A781D0008AB1F8881
:10A050000C000123022A18D14A68507811780002B6
:10A060002B4A0843801803280FD800F0C5FF0225AB
:10A070004439E06801F0F0F9C0B20723B84204D3D4
:10A080007B190193152B02DD0D231800FEBDE0683E
:10A090002A003100C01900F03FFF6B4600209B886A
:10A0A000E268D0541B4B1B68834203D01B68834279
:10A0B00000D098470023E8E70B23002FE5D1022DBD
:10A0C000E2D1737832781B021343E2681380114B9C
:10A0D0001B68002BEED01B68002BEBD00120E8E7BB
:10A0E0000B23002FD1D1062DCED12A003100E068FC
:10A0F00000F012FFDEE70B23002FC6D1012DC3D1E4
:10A1000032787533012AC0D8E3681A70D2E7C046A6
:10A1100000D6FFFF9069FF1F70B50C0015000728DF
:10A1200037D800F069FF041436361B36242E182069
:10A1300015290BD8184E16220021300000F034FFEC
:10A1400022002900300000F0E7FE002070BD18203A
:10A150000229FBD11288114B1A80F6E71820082932
:10A16000F4D10A000E48290000F096FFEDE7182010
:10A170000129EBD10B4B10780B49DA69FFF7DEFEB2
:10A18000E3E718200129E1D1064B10780749DA6B83
:10A19000F4E70220DAE7C0467869FF1F4245FF1F57
:10A1A0003845FF1FC844FF1FF044FF1F1045FF1F25
:10A1B000030010B50020DB0704D50721024A03483D
:10A1C00000F08CF810BDC046E4B70011C844FF1F72
:10A1D000054A03001068002803D082889A4201D102
:10A1E000806870470068F6E7946BFF1F0A880300D9
:10A1F00008009A4204D08A8804309A4200D0002095
:10A2000070470000F8B5F82200230D4F0D4E796815
:10A21000050042433370994200D07B600A4C002114
:10A22000200000F0C1FE00231A007C60AB4202D186
:10A2300000203370F8BD01332280DBB2F834F5E73B
:10A24000946CFF1F906CFF1F986BFF1F73B56B46DC
:10A2500001900600684615001980FCF743FF041EB4
:10A2600011D1002D0FD07689002E11D00C2000F0D6
:10A270002BFF00280ED0084A046013688680856092
:10A28000002B02D11060200076BD1A001B68F7E792
:10A290000224F8E71324F6E7946BFF1F0121002244
:10A2A0000A4B10B549420A4C198099809A719A70EC
:10A2B000084B2070012019805A60FFF7A3FF207817
:10A2C000FCF76EFF0448FDF719FF10BD9869FF1FEA
:10A2D0009C6CFF1F946CFF1F89A30011022310B513
:10A2E000002802D0FFF7B2FF0300180010BD0000E5
:10A2F000030010B50020DB0704D50421024A0348FF
:10A30000FFF7A4FF10BDC046F8B700114845FF1F76
:10A31000F0B50E2687B003930CAB1F8802ABF6187E
:10A320000500080031000292FDF75EF804000120EC
:10A33000002C0FD03088FFF74BFF03000E20002BBE
:10A3400008D05E68002E05D021002800039B029AE9
:10A350000097B04707B0F0BD0A4B10B5984207D13F
:10A360000122002352420A808B708A808B7110BDBB
:10A37000FFF73CFF0028FAD001235B420380002353
:10A380008370F4E7FFFF0000F8B5050001290AD14A
:10A39000134E00243388F827AB4219D02800114906
:10A3A000FFF7DAFF06E0022904D10139FDF724FFA7
:10A3B0000028EDD0F8BD3B0063437268D018D35A33
:10A3C000002B09D03A00002100F0EEFD0134E4B288
:10A3D000054B1B78A342EED801235B423380DDE7B7
:10A3E000946CFF1F9869FF1F906CFF1F10B5FFF75B
:10A3F000FDFE03000020834200D0987810BD0000CD
:10A40000F0B589B01C000EAB80CB03901E8810AB5A
:10A410001B78049202930B7A0D00DB0616D42B787E
:10A420000593022B24D00498FFF7D2FE002812D007
:10A4300003689C46002B0ED0029B2200019329004A
:10A440003B00644603980096A04705E00498FFF798
:10A45000BFFE002802D10E2009B0F0BD8368002B9A
:10A46000F9D00A222900039898470028D7D0F3E7AB
:10A470006B6858781A786B4B000210439842D2D818
:10A48000043B984210D2684B984242D015D8674B93
:10A49000C0180128C7D80B20002EDDD1EB681A7830
:10A4A00059683A80200028E0614BC018032800D981
:10A4B00079E000F0A1FD846A789E5E4B9842B2D1AB
:10A4C0000B20002EC8D101233B80EB6831001B78A4
:10A4D00023706889013080B2FCF786FF3A88031E3A
:10A4E0000ED0017802328A183A804289627042891D
:10A4F000120AA27059680278E01C00F00DFD06E017
:10A5000004323A8031000422601C00F04DFD00202E
:10A51000A2E70B20002E9FD1EB6807A91E88042319
:10A520003B80330A300026706370FCF75DFF051E28
:10A5300028D004AB9A890E2304A95B183E49C6684B
:10A54000FCF7C6FF00280BD12B783C486A680599B8
:10A55000FBF77CFB002803D1012304AA5B42D381D3
:10A560003278022A06D17168201D00F0D5FC3B88A4
:10A5700002333B800E2304AA9B181B88A3701B0A7E
:10A58000E370C4E704ABDE81F4E70B20002E00D0BB
:10A5900062E7E9680398FFF729FF02233B802070F8
:10A5A000000A6070B3E70B20002E00D054E70222AF
:10A5B000EB681B883A8023701B0A6370A7E7E86882
:10A5C00000F04AFFC2B203000720B24200D243E7C4
:10A5D0000DD00299DBB27118994202DB921BD3B203
:10A5E0000293029BE9681A003B8089195AE700230D
:10A5F000F6E70B20002E00D02EE70722EB683A800A
:10A600001A7822705A7862705A88A2705A88120A90
:10A61000E2701A792271DA886271DB881B0AA371F1
:10A6200075E7C046042900000228000000D8FFFF9B
:10A63000FFD6FFFF03280000FFFF000028B700112E
:10A64000F0B58DB06B460020089120229B5E8342BE
:10A650003DDAA64B187800F037FC071E32D003789D
:10A66000B02B2CD10079023816281FD800F03CFC02
:10A6700017001E001E001E0031001E0096001E0066
:10A680001D011E0052011E0073011E00CD011E009F
:10A6900050021E001E001E008E021E00E302944B9C
:10A6A00094491B8878880B80FBF710F83800FCF77A
:10A6B00081FF914B1B68002B01D038009847380070
:10A6C00000F0DAFD8020089B0002434018000DB026
:10A6D000F0BDF6220021874800F066FC0BAA3B7B08
:10A6E0007989388900923A000D32FCF795FD040013
:10A6F000804B1B78002C3FD146E0804B7888059337
:10A700007F4B4100CB5A0BAE073BDBB23288029342
:10A71000002301937B4B210006930093059BFFF7D9
:10A720006FFE744D002810D1069B3A8A1B889A420E
:10A730000BD138000599123000F066FC002804D0D7
:10A740002B7862899B00EB185A80162306A81B18E9
:10A75000328820007989FCF7BBFE2B7804009A0030
:10A76000AA1851880029C3D00133DBB22B7000280E
:10A7700007D006A9C98A9180634A12889A42BCD838
:10A7800002E0012149429180002B04D05949788888
:10A79000FAF7D0FF8AE73E890A2479E000253E894E
:10A7A000574B06937B88069A5B009B5A033B9D425E
:10A7B00002DB002DF0D05BE0162206A812183B7BCE
:10A7C000798900923A0030000D32FCF725FD0590A2
:10A7D000002858D04689017A7888FCF7E7FC041EE7
:10A7E00044D1464B78880793069B4100C95A454B94
:10A7F0000439C9B206AAD28A069302910194009341
:10A800000599079BFFF7FCFD041E2FD1069B3949D4
:10A810001A88931C002D26D14B807988384B49002B
:10A82000CB5A5119033B8B4220DD059B31485B8994
:10A8300041190B71A91C0135C9B2EDB20591451939
:10A840001B0A2B71059B2D490433181800F064FB7B
:10A850002C4B059A1B88D318DDB22C4B9E4205D099
:10A860000136B6B29CE749889942D6D0002D0CD06B
:10A87000204C2800618800F0F7FA207021007888C9
:10A88000FAF768FF12E7059CF0E7002C00D183E798
:10A890007B78142B00D109E716493B794E800B7069
:10A8A0000C717888FAF708FF00E7162406ABE41865
:10A8B00021003889FCF798FD011E00D1B7E17888A6
:10A8C00022880F4C45002C5B0A4D013CE4B20294F7
:10A8D00000240F4B01940095FFF792FD041E00D059
:10A8E00014E129007888FAF745FFDFE69C6CFF1F2A
:10A8F0003444FF1FA069FF1F9469FF1F9A6AFF1F5E
:10A90000D065FF1F906BFF1F3244FF1FFFFF000049
:10A91000A269FF1F162406ABE41821003889FCF752
:10A9200063FD011E00D182E178882288AE4C45008B
:10A930002C5BAE4D013CE4B202947C89AC4B01949B
:10A940000095FFF75DFD041E00D0DFE02900788848
:10A95000FAF71AFFAAE60025A44B1D803B00FE3340
:10A960001B78A24A78880792AB4208D99E4B12887E
:10A970000693069943005B5A013B9A4203DB079911
:10A98000FAF70CFF92E616246B00FB18059306AB52
:10A99000E418059B21001889FCF726FD011E03D150
:10A9A000059B01241E8973E77888924B2288069CB8
:10A9B000099343001B5B904E013BDBB202930023E3
:10A9C00000960193099BFFF71BFD041E02D0059B17
:10A9D0001E895DE77B88069A5B009B5A079A108860
:10A9E00032881218934202DC1B1A013B33807F4CE1
:10A9F000023032880999001900F08EFA23883288D3
:10AA000001359B182380EDB2A8E70BAA3B7B79891F
:10AA1000388900923A000D32FCF7FEFB00250590C4
:10AA2000059B002B04D10A24002D00D16EE060E0CC
:10AA3000059B7888197AFCF7B9FB0100041E63D1E5
:10AA4000694C6C4B788806940993069B4400E45A41
:10AA5000694B063CE4B20BAE328807930294019135
:10AA600000930599099BFFF7CBFC041E4CD1079B73
:10AA70005E491B881A1D002D30D14A80059B5B4C16
:10AA80005A8963191A716B1C9BB2E318120A1A7166
:10AA9000162306A832881B1879890598FCF718FD3B
:10AAA000FF21AA1C2E1D03350B00059092B2B6B2F1
:10AAB000ADB2002803D006ABDB8AD9B21B0AA218BC
:10AAC000651911712B714C4D301D2A884949201888
:10AAD00000F022FA2B88F618B5B2A1E74988914216
:10AAE00007D17A8806995200525AEB18053A9A42D1
:10AAF000C4DC3E4C2800618800F076FB2070210009
:10AB00007888FAF755FED1E5002DF2D13E89BFE6EF
:10AB1000162606ABF61831003889FCF765FC3D00B7
:10AB20000400FF3500282DD0037A9B060CD40022A8
:10AB30007B893989788800923A000C32FFF7E8FB6C
:10AB4000041E10D03E8915E03088FFF741FB002835
:10AB50001AD08368002B17D02100122278889847DA
:10AB6000041EE4D0EEE7AB78002B02D17888FAF728
:10AB70002FFE0026AB78002B00D097E5002C00D1EB
:10AB800094E585E60124DDE70E24DBE7162506AB18
:10AB9000ED1829003889FCF727FC041E47D0037AFA
:10ABA0009B0611D4154A7B881188994203D014481A
:10ABB000814207D11380134BF8261D780023D9B2A8
:10ABC000A94221D30924A1E72888FFF701FB002827
:10ABD0002FD08368002B2CD0210012227888984730
:10ABE000041EDFD092E7C046D065FF1FA069FF1F9B
:10ABF000A269FF1F9A6AFF1F906BFF1F946CFF1FD3
:10AC0000FFFF0000906CFF1F31005943546801336F
:10AC10006018615A0029D2D13C0008342100F82282
:10AC200000F07AF921007888FAF7DAFD3EE5012490
:10AC30006CE70E246AE71D4B1A887B889A4231D054
:10AC40007888FAF7D7FD31E5F82305985168434332
:10AC5000CD18C95A00291FD03B7A012B0BD16C8823
:10AC6000AB887888AA1D0094FFF752FB041E02D01F
:10AC700000233B722E88F8220021280000F094F96E
:10AC800000232B80059B0133DBB20593084B05990C
:10AC90001B78064A8B42D7D801235B421380002CD5
:10ACA000CED0F5E5002634000596EFE7946CFF1F43
:10ACB000906CFF1F70B504000E001500FFF796FAA8
:10ACC000031E08D131000548FFF790FA0300112058
:10ACD000002B02D01C8000209D7070BDFFFF000083
:10ACE000F8B50B4F06003B780D001400FF2B0ED07B
:10ACF0000A2000F051F9011E09D0B123038000237E
:10AD000046800371C5800481387800F0D5FAF8BD1B
:10AD10008945FF1FF7B50F0008A90600088809A993
:10AD20000B240988002821D10234022B1ED155782A
:10AD300013782D021D432B008B4301937334002B9A
:10AD400014D1FB68300019000093FFF74FFB019C02
:10AD500085420BD02A0030000099FFF7ABFF041E9C
:10AD600004D12A0030007989FFF7BAFF2000FEBD28
:10AD7000F0B50E7885B003900AA805880120022E50
:10AD80000DD14C682778647824023C43054FBC42BF
:10AD900005D10398DBB201960095FFF7BBFF05B024
:10ADA000F0BDC0460229000010B504000C4800F0B8
:10ADB0006BF90C48A16B00F067F90B48E16B00F0F0
:10ADC00063F90A48216C00F05FF9094B09481968DA
:10ADD00000F05AF9084B1B68002B00D09847FEE79B
:10ADE000FAB5001110B600111FB600112EB60011F1
:10ADF00004ED00E03DB60011A06CFF1F002307B575
:10AE000001A80193FFF7D0FF044A0548002110B5BF
:10AE1000121A00F0C9F8F8F79DFDFEE7A46CFF1FB9
:10AE20008C45FF1F0000000001B40248844601BCAD
:10AE3000604700BF5522000001B40248844601BCAF
:10AE4000604700BF055E000001B40248844601BCB3
:10AE5000604700BFC926000001B40248844601BC17
:10AE6000604700BF5539FF1F01B40248844601BC4A
:10AE7000604700BF350E000001B40248844601BCA3
:10AE8000604700BF0D52010001B40248844601BC76
:10AE9000604700BFD949010001B40248844601BCA3
:10AEA000604700BF6DBC000001B40248844601BC8D
:10AEB000604700BF017F000001B40248844601BC26
:10AEC000604700BFC94A010001B40248844601BC82
:10AED000604700BFF54E010001B40248844601BC42
:10AEE000604700BF1147010001B40248844601BC1D
:10AEF000604700BF6D3CFF1F01B40248844601BC9F
:10AF0000604700BF1D3BFF1F01B40248844601BCDF
:10AF1000604700BF9DA9000001B40248844601BCFF
:10AF2000604700BFE94C010001B40248844601BCFF
:10AF3000604700BFDD30FF1F01B40248844601BCFA
:10AF4000604700BF9135FF1F01B40248844601BC31
:10AF5000604700BF0124000001B40248844601BCE0
:10AF6000604700BFC9A9000001B40248844601BC83
:10AF7000604700BF311B000001B40248844601BC99
:10AF8000604700BF9938FF1F01B40248844601BCE6
:10AF9000604700BF8D3AFF1F01B40248844601BCE0
:10AFA000604700BF1D4D010001B40248844601BC4A
:10AFB000604700BF154D010001B40248844601BC42
:10AFC000604700BFC521000001B40248844601BCAF
:10AFD000604700BF8552010001B40248844601BCAD
:10AFE000604700BFC56D010001B40248844601BC42
:10AFF000604700BF014C010001B40248844601BC17
:10B00000604700BF593CFF1F01B40248844601BCA1
:10B01000604700BFCD4C010001B40248844601BC2A
:10B02000604700BF5952010001B40248844601BC88
:10B03000604700BFA139FF1F01B40248844601BC2C
:10B04000604700BF6932FF1F01B40248844601BC5B
:10B05000604700BF456B010001B40248844601BC53
:10B06000604700BF3555000001B40248844601BC6A
:10B07000604700BF091B000001B40248844601BCC0
:10B08000604700BF493BFF1F01B40248844601BC32
:10B09000604700BFE53A010001B40248844601BCA4
:10B0A000604700BF810E000001B40248844601BC25
:10B0B000604700BF1D4B010001B40248844601BC3B
:10B0C000604700BFC132FF1F01B40248844601BC83
:10B0D000604700BF3D4B010001B40248844601BCFB
:10B0E000604700BFE117000001B40248844601BC7C
:10B0F000604700BF090E000001B40248844601BC4D
:10B10000604700BF851F000001B40248844601BCAF
:10B11000604700BF691F000001B40248844601BCBB
:10B12000604700BFD91B000001B40248844601BC3F
:10B13000604700BFE537FF1F01B40248844601BCE9
:10B14000604700BF093BFF1F01B40248844601BCB1
:10B15000604700BF8D12000001B40248844601BC64
:10B16000604700BFC95C010001B40248844601BCCD
:10B17000604700BFB54C010001B40248844601BCE1
:10B18000604700BFB70E000001B40248844601BC0E
:10B19000604700BF5147010001B40248844601BC2A
:10B1A000604700BFB14E000001B40248844601BCB4
:10B1B000604700BFC51D000001B40248844601BCC1
:10B1C000604700BFA946010001B40248844601BCA3
:10B1D000604700BF7D18FF1F01B40248844601BCD0
:10B1E000604700BF4D1F000001B40248844601BC07
:10B1F000604700BF090E000001B40248844601BC4C
:10B20000604700BF75A9000001B40248844601BC34
:10B21000604700BF2124000001B40248844601BCFD
:10B22000604700BF2951010001B40248844601BCB7
:10B23000604700BF1537FF1F01B40248844601BCB8
:10B24000604700BF7918000001B40248844601BC81
:10B25000604700BFE1AC000001B40248844601BC75
:10B26000604700BF453CFF1F01B40248844601BC53
:10B27000604700BF4550000001B40248844601BC4D
:10B28000604700BF434D010001B40248844601BC41
:10B29000604700BF5549010001B40248844601BC23
:10B2A000604700BFF30E000001B40248844601BCB1
:10B2B000604700BF8B52010001B40248844601BCC4
:10B2C000604700BF594F010001B40248844601BCE9
:10B2D000604700BFADAE000001B40248844601BC27
:10B2E000604700BF0134FF1F01B40248844601BC1F
:10B2F000604700BF2146010001B40248844601BCFA
:10B30000604700BFF94C010001B40248844601BC0B
:10B31000604700BF213AFF1F01B40248844601BCC8
:10B32000604700BFC53F000001B40248844601BC2D
:10B33000604700BFE548000001B40248844601BCF4
:10B34000604700BF5125000001B40248844601BC9B
:10B35000604700BF3D18000001B40248844601BCAC
:10B36000604700BFE139FF1F01B40248844601BCB9
:10B37000604700BFD1A5000001B40248844601BC6B
:10B38000604700BF9130FF1F01B40248844601BCF2
:10B39000604700BF2526000001B40248844601BC76
:10B3A000604700BF0189000001B40248844601BC27
:10B3B000604700BFB352010001B40248844601BC9B
:10B3C000604700BF151BFF1F01B40248844601BC43
:10B3D000604700BF6939FF1F01B40248844601BCC1
:10B3E000604700BF5D17000001B40248844601BCFD
:10B3F000604700BF056A000001B40248844601BCF2
:10B40000604700BFA134FF1F01B40248844601BC5D
:10B41000604700BFE928000001B40248844601BC2F
:10B42000604700BF0933FF1F01B40248844601BCD6
:10B43000604700BF291C000001B40248844601BCDB
:10B44000604700BF5118FF1F01B40248844601BC89
:10B45000604700BF8132FF1F01B40248844601BC2F
:10B46000604700BFDD52010001B40248844601BCC0
:10B47000604700BFA54F010001B40248844601BCEB
:10B48000604700BFF136FF1F01B40248844601BC8B
:10B49000604700BFEDA5000001B40248844601BC2E
:10B4A000604700BFED4A010001B40248844601BC78
:10B4B000604700BF4551010001B40248844601BC09
:10B4C000604700BF6571010001B40248844601BCB9
:08B4D000604700BF4134FF1F7B
:10B4D8000002010302030303040305020602070234
:10B4E800080209000A030B030C020D020E030F03E6
:10B4F800100311031303140315001600313D001146
:10B50800653D001100000000020000001AB500119E
:10B51800192A0F180A000000F1590000FD24000044
:10B528004146010005780011199800118D6C001131
:10B5380009760011454E001141A60011054B001176
:10B54800E53F0011F93E0011000000001E1E00003A
:10B558000200000064B50011F4FFF3FFF0FF0000E3
:10B5680015410011000000000000000054757961C9
:10B578000056302E360030303031006769746875F7
:10B58800622E636F6D2F70767678004254483031A2
:10B598000000000002000000B0B50011292A282A86
:10B5A800272A262A252A242A0A180000E20400004D
:10B5B8007102000078EC00007440000010270000C1
:10B5C80060F00000000000001F501D000206B400DB
:10B5D80030313233343536373839414243444546C1
:10B5E800005048592B36325858504C555330353046
:10B5F80034005B48617264206661756C7420686110
:10B608006E646C65725D0A004C522020203D20302B
:10B6180078253038780A0050432020203D203078A3
:10B62800253038780A0050535220203D20307825A4
:10B638003038780A0049435352203D20307825306D
:10B6480038780A0055520011A95200110000000074
:10B658000200000064B600116F2A6E2A1A18000052
:10B6680001A00000000000006410B71DC8206E3B58
:10B67800AC30D9269041DC76F4516B6B5861B24DF1
:10B688003C7105502083B8ED44930FF0E8A3D6D65B
:10B698008CB361CBB0C2649BD4D2D38678E20AA0C3
:10B6A8001CF2BDBDFB349B5F8000008000100000D1
:10B6B800000000008F580011196F0011B3580011D5
:10B6C8002173001137590011F7720011AD5900119B
:10B6D800CD720011FF59001195740011675A0011BD
:10B6E80095740011995A00114F740011AD59001149
:10B6F80085720011255A00112D74001100000000F8
:10B70800000000000B5B00112D7400116D5B00112F
:10B71800316F0011052A042A012A002A0229032868
:10B72800012800280118001800000000000000008F
:10B73800000000000000008701010201020101026F
:10B7480001020303040103010101010103030201D2
:10B7580003000D000E001000110013001401070172
:10B7680008010A010B011C011D020402050207025F
:10B77800080219021A021C021D0301030203170022
:10B788000201000504000807000B0A001716001D37
:10B798001C010201010504010E0D01111001141311
:10B7A800011716011A19020201020B0A020E0D02F4
:10B7B8001110021413021716030504030807030BDC
:10B7C8000A030E0D0001020307090A0B0E0F1011E0
:10B7D80012141718191A1B1F20212200899F001103
:10B7E80045A0001100000000020000002EB7001163
:10B7F8000000000071AD0011000000000200000010
:04B808002CB7001148
:020000041FFFDC
:10000000000000008D3E001120B500111CB500114C
:100010009862FF1F000000000000000000000000C8
:1000200000000000000000000000000000000000D0
:1000300000000000000000000000000000000000C0
:1000400000000000000000000000000000000000B0
:1000500000000000000000000000000000000000A0
:100060000000000000000000000000000000000090
:100070000000000000000000000000000000000080
:100080000000000000000000000000000000000070
:100090000000000000000000000000000000000060
:1000A0000000000000000000000000000000000050
:1000B0000000000000000000000000000000000040
:1000C0000000000000000000000000000000000030
:1000D0000000000000000000000000000000000020
:1000E0000000000000000000000000000000000010
:1000F0000000000000000000000000000000000000
:1001000000000000000000000000000000000000EF
:1001100000000000000000000000000000000000DF
:1001200000000000000000000000000000000000CF
:1001300000000000000000000000000000000000BF
:1001400000000000000000000000000000000000AF
:10015000000000000000000000000000000000009F
:10016000000000000000000000000000000000008F
:10017000000000000000000000000000000000007F
:10018000000000000000000000000000000000006F
:100190006534FF1F5533FF1FC166010000000000DA
:1001A000000000000000000000000000000000004F
:1001B000000000000000000000000000000000003F
:1001C000000000000000000000000000000000002F
:1001D000000000000000000000000000000000001F
:1001E000000000000000000000000000000000000F
:1001F00000000000000000000000000000000000FF
:1002000000000000000000000000000000000000EE
:1002100000000000000000000000000000000000DE
:1002200000000000000000000000000000000000CE
:1002300000000000000000000000000000000000BE
:1002400000000000000000000000000000000000AE
:10025000000000000000000000000000000000009E
:10026000000000000000000000000000000000008E
:10027000000000000000000000000000000000007E
:10028000000000000000000000000000000000006E
:10029000000000000000000000000000000000005E
:1002A000000000000000000000000000000000004E
:1002B000000000000000000000000000000000003E
:1002C000000000000000000000000000000000002E
:1002D000000000000000000000000000000000001E
:1002E000000000000000000000000000000000000E
:1002F00000000000000000000000000000000000FE
:1003000000000000000000000000000000000000ED
:1003100000000000000000000000000000000000DD
:1003200000000000000000000000000000000000CD
:1003300000000000000000000000000000000000BD
:1003400000000000000000000000000000000000AD
:10035000000000000000000000000000000000009D
:10036000000000000000000000000000000000008D
:10037000FDAD0011000000000000000000000000C2
:10038000000000000000000000000000000000006D
:10039000000000000000000000000000000000005D
:1003A000000000000000000000000000951AFF1F80
:1003B000000000000000000000000000000000003D
:1003C000000000000000000000000000000000002D
:1003D000000000000000000000000000000000001D
:1003E000000000000000000000000000000000000D
:1003F00000000000000000000000000000000000FD
:08183800B070FF1F4118FF1FF3
:10184000024981F3088802F063FC0000B070FF1FBA
:1018500010B502F01DFA072804D0122808D002287B
:1018600008D010BD044A0420136B01331363F8E75A
:101870000220F6E71420F4E77866FF1FF8B50700AA
:101880000C0026002500503630785135002804D150
:101890000300287058342370F8BD2978CA00481E08
:1018A0008141A3183800A25C5B68C9B2FFF7D0FF82
:1018B00000280DD12B78DA00A218013350602B706C
:1018C0003378044A013B3370136A01331362D8E75B
:1018D0000123DFE77866FF1F5C234343074910B508
:1018E000C9180B0058331B78012B05D1FFF7C6FF31
:1018F000034A936A0133936210BDC046AC66FF1F72
:101900007866FF1F10B502F0EBFA064A01211300BA
:1019100010CB4942D967044B136002F0B1FB2000A1
:1019200010BDC04600E100E01000100010B504003A
:1019300002F0D6FA024B1C6002F0A2FB10BDC046BA
:1019400000E100E010B5040002F0CAFA4021094AA3
:10195000200013688B43136002F0EAF901F064FD84
:101960000022054B01201A60044B04321A6002F079
:1019700037FAFEE71CF00040C4F00040C0F0004021
:10198000431E5A425341A022F0B5D2015B4213409C
:10199000154D164A40019B182A18127E8BB00191F2
:1019A000002A1BD01A000832D46F0022E6B206AF1C
:1019B000E4B294420EDC2818C369002B08D00199C8
:1019C00002AA117106AA049202AA167303A89847E4
:1019D0000BB0F0BD1978B9540132EAE71A7D1A78D4
:1019E00006AB01261A70E6E73869FF1F0040004089
:1019F000F0B5254B04004001C25C85B0002A2BD015
:101A00001A18117E002927D0917E002924D011793F
:101A1000022921D11689D788D168F51BADB22A1CBD
:101A2000102D00D9102292B2BE4217D118180123EE
:101A300003710023C269C38003819A4206D06846BD
:101A4000032103730171029301A890470820002C21
:101A500000D0192001F034FC05B0F0BD013C654216
:101A60006C41A0256442ED012C40084D1B186419FF
:101A7000074D0633013A92B2AA42EDD01888461CAF
:101A80001E80085C2070F5E73869FF1F00400040A9
:101A9000FFFF00000F220E4B10B59868104002386F
:101AA0000A280BD802F0D8F80D0A0B0A0A110A0A04
:101AB0000A0A060002210020FFF762FF10BD012183
:101AC000F9E70020FFF794FFF8E7DB6FF6E7C04681
:101AD000004000400F220E4B10B5986810400238AD
:101AE0000A280BD802F0B8F80E0A0B0A0A120A0AE2
:101AF0000A0A060002210120FFF742FF10BD012162
:101B00000800F9E70120FFF773FFF7E7DB6FF5E760
:101B10000090004013B5334C2378072B3DD8324B4F
:101B20001A78324B002A39D18022196852020A43AE
:101B30001A60252001F034FF20232D4A11680B4341
:101B4000802113606B460422C905086807331042E0
:101B500028D080210422C905C86810422ED08021D7
:101B60002020C905CA688243CA6014221A701A78F4
:101B7000002A2FD18021C905C86820320243CA60DB
:101B800014221A701A78002A28D11A4B1A7D22784A
:101B90005A601D221A705932DA6013BD1A6816494C
:101BA0000A40C5E7086802430A6014221A701A78CE
:101BB000002ACED01A78013AD2B2F7E7C8680243B9
:101BC000CA6014221A7019784A1ED2B21A700029FB
:101BD000F9D1C4E71A78013AD2B2C7E71A78013AC4
:101BE000D2B2CEE7C444FF1F8C45FF1F3CF000403B
:101BF000BC44FF1F00200040FFFFFEFF564B70B5A6
:101C00001B68012B03D1554A936D0133936502F094
:101C10001FF9534B534A1860534B544C1A6001231D
:101C2000534A1360534A13602378002B06D00622D0
:101C30005149524802F054F800232370504A514B46
:101C400010681B78C1B2002B0ED14F4CC0B2237864
:101C50005BB2002B4FDB237824785BB264B21B04A9
:101C600024021B191B1813600B1C50294ED950233A
:101C7000464A47491078DBB2FF2202284BD1086858
:101C8000444C454D267890432A78964254D9227880
:101C900024782E78023B5D10A31B6B435201D31AAC
:101CA00010335B111843086002F052F9031F012B37
:101CB00045D83A4B1B78002B06D0394B1B78002BAC
:101CC00002D0002002F014FAA122364B920099783B
:101CD000354B4A431B689B18832292009B181B7844
:101CE000033B012B03D8AF20400002F079F9012219
:101CF0002E4BDA8270BD237824785BB264B2FF3356
:101D0000FF341B0424021B190138ABE7CAB2022AB4
:101D1000AED20223ACE70868254C264D26789043C6
:101D20002A78964208D9227824782D78023B5B10D5
:101D3000641B63435201B2E72378DBB2B2E70228A7
:101D4000D5D11D4B1B78013B022B03D91B4B1B78B4
:101D5000022BCCD16C20C8E79809FF1FFC0FFF1F96
:101D6000B065FF1FFF3F000014100340B465FF1F64
:101D70000C10034000100340D50BFF1F7211FF1F12
:101D8000B40003408C09FF1F680AFF1F490AFF1FA8
:101D900094000340460AFF1F470AFF1FF908FF1F70
:101DA0002209FF1F300DFF1F3409FF1FBC0BFF1F4F
:101DB000440AFF1F450AFF1F1C09FF1F2309FF1FBD
:101DC00010B501F0EDFF0022014B1A8010BDC04696
:101DD000AC65FF1F10B502F0B3F8A121054A8900D8
:101DE0009478054A61431268044B5218528C1A8049
:101DF00010BDC046300DFF1F3409FF1FAC65FF1F2B
:101E000010B50D4B0D4A9978A1239B004B431268E6
:101E1000D218531DD97F0A4B1B88994209D2441C02
:101E200007D0C82805D0D2695B1A5A43054B5343E3
:101E3000C01801F065FF10BD300DFF1F3409FF1FF2
:101E4000AC65FF1F7102000070B5244D2B68002B9C
:101E500028D001F085FF2B68D8402B680400002BA8
:101E600027D001F0EDFF2B68D8401D4B1D4A997813
:101E7000A1239B004B431268D118D25C91239B0095
:101E8000002A20D0CA580132CA50174B17491B6884
:101E90000868834214D3D23B181A012A1AD0144B73
:101EA000186070BD01F05CFF124B196801F048FF2B
:101EB000D3E701F0C5FF0F4B196801F041FFD4E7EC
:101EC0000D495B18E8E7CA500C4B1B68DB68E41847
:101ED000201AE4E7F530FF30E1E7C0461C08FF1F99
:101EE000300DFF1F3409FF1F9C09FF1FB065FF1F46
:101EF000A009FF1F1808FF1F2DFF3F00B865FF1F37
:101F000070B504000D00282916D10300A433C2883F
:101F10001B889B1A0B4A9BB293420DD906006A3666
:101F200005223100653002F0B3F8002804D13100F9
:101F3000200002F0C5F870BD2900200002F030F941
:101F4000F9E7C046FE7F0000F8B50400012001F06B
:101F50006FFF02F02DF8174A174910600968030057
:101F60001648174E01601748776805680020AF4291
:101F700001D27068281A144D091928601348C162EB
:101F8000A421446A49032143416211490978002987
:101F900005D010490978022902D10F3B1360F8BD22
:101FA000012901D1083BF9E7032901D1053BF5E7F8
:101FB000033BF3E7E408FF1F28F00040340AFF1F4B
:101FC00028100040180AFF1F1C0AFF1F00F00040E5
:101FD0001C09FF1F4A0AFF1F70B580241025E40565
:101FE000A3682B43A36001F073FFA368AB43A36016
:101FF00070BD0000F7B5160080221C001023D2052A
:102000000191916805000B43936000225A4BD73031
:102010001A6002F0B5F89D232A002F009B00EB58B0
:10202000CA3201210092FC37002B01D00021009A16
:10203000386802F0BDF82900009BCB311A784F4B6D
:10204000D3351A604B780A781B0213438A7812043E
:102050001A43CB781B061343494A1BBA13604B79CA
:102060000A791B0213438A7912041A43CB7931008F
:102070001B061343434A1BBA13606B782A781B0272
:102080001343AA7812041A43EB781B0613433E4A03
:102090001BBA1360019A330213433C4A13603C4B52
:1020A00022001B1B9C4603293DDCB3089A00130049
:1020B0005142B21A032A46D1354AE018511A8278A1
:1020C0004078120400020243E05C043302430A60D9
:1020D0000022FF2B4BDDF0222E4B12011A600F2243
:1020E0002D4B1A602D4A1368002BFCD00023224A86
:1020F00027491360091B321D0B191B68043A180A83
:1021000023706070180C1B0EA070E3700434002A5A
:10211000F2DC802210213B68D20501333B609368DA
:102120008B439360F7BD6346D578981893782D0656
:102130001B042B43157804392B43557804322D02A8
:102140002B430360AFE7022A0AD1114AE05C511A1F
:10215000E2185278120202430A6004339BB2B7E7D6
:10216000012AB5D10A4A521AE15C1160F5E7084923
:1021700059180A600433ACE7000004403C000440F6
:102180003800044034000440300004400C00044097
:102190000001044004000440100004401400044006
:1021A000F7B5150080221C001023D205009191681C
:1021B00007000B4393600023654AD730136001F09A
:1021C000DFFF9D233E009B00F9583B00CA363200DA
:1021D000FC33002900D07FE0586801F0E9FF3900A6
:1021E00032785C4BCB311A604B780A781B02134370
:1021F0008A78AC4612041A43CB78281D1B06134379
:10220000554A1BBA13604B790A791B0213438A792A
:1022100012041A43CB791B061343504A1BBA1360AE
:102220004B7A0A7A1B0213438A7A12041A43CB7A36
:1022300021001B0613434A4A1BBA1360009A2B0263
:102240001343484A13602200474B1B1B0093009B1B
:10225000CE785B1801938B7836061B0433430E78D7
:10226000043833434E78043136023343019E3360E1
:102270000328ECDC0321A808431C9B0029408000B4
:1022800003292BD13849E5185E18A9786D78E35CED
:1022900009042D022943194331600300083300214A
:1022A000FF2B2DDD314B324919600F21314B196065
:1022B000012327490B60304B19680029FCD0062107
:1022C0001B680B40042B20D080220020D20593688D
:1022D0000A318B439360FEBD01217DE7022908D1BD
:1022E00021495D18E1184978E35C09021943296026
:1022F000D3E70129D3D11C495918E35C0B60CCE723
:102300001948181801600433CAE7002310490B600C
:102310006346002B0CDC3B00FC335A681021013271
:102320005A608022D205936801208B439360D2E7E4
:10233000009B9B181B68190A13705170190C1B0E17
:10234000D37004235B4291709C440432E0E7C046A2
:10235000000004403C0004403800044034000440C5
:10236000300004400C00044000010440040004401C
:10237000080F0000100004401400044070B5061E51
:1023800019D00222614B9B799343012B13D1604BEF
:102390001A78FF2A0FD15A78FF2A0CD19A78FF2A8F
:1023A00009D1DA78FF2A06D11A79FF2A03D15B799D
:1023B000FF2B00D1A7E0574B0C201A78012A08D038
:1023C0000022554D1A702B781A00093A042A01D8B8
:1023D000212070BD5A1F012AFAD94C4CA07B042839
:1023E00000D990E0A279032A00D98CE0821E012A4C
:1023F00003D862881F2A00D885E0002E61D0012E04
:1024000000D080E0A288012AE2D0002B0AD1013856
:10241000032803D801F020FC151D19151F202E706C
:1024200001F0B6FC2B785A1E032A16D800253B4B28
:102430001D602823237501F0BBFCA8422ED0A58087
:10244000C6E7022320202B70EAE7042322202B700A
:10245000E6E7032321202B70E2E7073B012BB7D8E7
:102460002F4B1B68DB6A9B06B2D52E4B1A78002ACD
:10247000AED1A27B911E012901D9002AA8D1022246
:1024800080211A702823284D89012878237501F0AE
:10249000BFFC80212878890101F002FE0123A3807E
:1024A000224B1B78002B0AD0FA228021204B92006D
:1024B0001B8809025A431C4B187801F099FC002034
:1024C00087E701F00DFD2B78A680073B012B06D98D
:1024D00018482E7001F00CFC1E2001F059FC114B25
:1024E000114C1A78002A06D0802100222078890118
:1024F0001A7001F08DFC01F0C3FD802120780902E3
:1025000001F086FCDBE7122063E7C046A60BFF1F45
:102510006B09FF1F1A09FF1F1C09FF1F4809FF1F36
:10252000B865FF1F2309FF1F1B09FF1F2109FF1F9C
:102530002C09FF1F0010004010B5002901D001F048
:10254000C7FB10BDF7B5604B01919978A1239B00A3
:102550004B435E4A060014681022E418D6235B0041
:10256000E0583623FF33E35C00279343222B41D10D
:10257000574B0F3A1A600760012501F0F9FC019BE7
:102580001880E8235B00E35C002B01D0B34258DDE8
:102590000023504FFB70AD33FF33E3581A68002A15
:1025A00003D09B88DB439B071DD03823FF33E35CBC
:1025B000002B18D09B235B00E35C002B13D1D1339D
:1025C000FF33E35CB3420EDAA4235B00E15AE01868
:1025D000090A023101F0ACFD23000122FE33013E65
:1025E00001351A87FA70E8235B00E35C002B2AD0E0
:1025F000A8B2FEBD03683D00002BBED08188043028
:10260000090A023101F094FDD6235B00E3581F60F4
:10261000B2E72300B133BA00FF33985801378188FD
:102620000430090A023101F083FDE8235B00E35C1A
:10263000BB42EEDCE822F61AED1800235200A35448
:10264000A6E70027F1E7200001F02AFB00281FD0B1
:10265000002E1DDD7319882647190193B60020004E
:1026600001F06EFD5A3080002018406801358188E5
:102670000430090A023101F05BFD200001F0D8FCB2
:10268000A3590133A351BD4202D0019B9D42E6D123
:10269000114BE35C002BABD095239B00E35C002B3C
:1026A000A6D00E4BE15A0029A2D00D4AA35C994254
:1026B00002D90133A3549BE700231A212000A3541D
:1026C00001F0AEFC94E7C046300DFF1F3409FF1F38
:1026D00000140340E010FF1F5A02000072020000C5
:1026E0005E020000F8B51D4B1D4F1A78002A10D16C
:1026F000BA7B002A02D101321A7003E0032AFAD011
:10270000022AF8D001F054FB00220120154B1A7068
:10271000F8BD154B154D1C68154B9E7801232B7089
:102720002878C0B200F0DEFCBB7B002B0BD101F09F
:1027300017FCA1239B007343E41883239B00E41838
:1027400023782B70E4E7032B02D101F0D9FCF0E7EA
:102750000020022BDCD101F0E3FCEAE71C09FF1F9B
:10276000A60BFF1F2309FF1F3409FF1F490AFF1F84
:10277000300DFF1FF0B587B00EAD2F780FAD2D785F
:102780000593AC46634614000E4D0CAA12782E78C1
:1027900003930D9B009201932200059B029701F089
:1027A000C7FB2E70012C01D0042C08D180220649D1
:1027B0008B889343054A1278D20113438B8007B06C
:1027C000F0BDC0461C09FF1F6C11FF1F7809FF1FD9
:1027D0000B001B3B70B504003020E02B0DD813001C
:1027E000E025493BFF3B9BB2ED00AB4205D8034BD4
:1027F000200019825A8201F093FB70BD8410FF1FE4
:1028000010B501F025FB054B00205B68052B04D9B2
:10281000034A5268D20200D4980810BD001000404C
:10282000FCE100E070B501F05BFB0D4B1B68FC3375
:10283000DC691D6AFFF7E4FF6419844204D2094B86
:1028400001241B68002B07D004220024064B1A70B9
:10285000064A93690133936101F012FC200070BDB8
:10286000B865FF1F9809FF1F2309FF1FFC0FFF1FFB
:1028700070B50C4D2B68FC335C6A01F031FBFFF73F
:10288000BFFF2B680025FC339B6AE318834204D208
:10289000054B1B68AB4200D1051B01F0F1FB280082
:1028A00070BDC046B865FF1F9809FF1FD722044BB3
:1028B00092009B5810B5002B00D0984710BDC04621
:1028C0000000FF1FF0B587B001F050F9FFF7EEFFF1
:1028D000CA4BCB4C04931B78022B45D1C94B1B68C8
:1028E000186A01F0A5FAC84BC84A1A60C84BC94A11
:1028F0001A60A022C84B52001A60049B187801F09D
:1029000037FCC649C64801F0ABFBC649C64801F0D2
:10291000A7FB1022C54BFF201A60802252031A60C9
:10292000802292031A60802212041A6001F0E0FBF8
:10293000012001F0A5F9FA20400001F0F1F958203A
:1029400001F04EFBBA4801F093FB012001F078FB47
:10295000072001F0DDFA2268B64B1A4084235B00A1
:102960001343236007B0F0BD01F07AFAB24E029033
:10297000322001F05DFA33681B0629D43C2001F0B7
:1029800057FA0F2001F054FA9C4B1B78012B00D111
:102990001EE180223368A94D134200D0A7E02B68C6
:1029A000032013432B6001F043FA01F059FA029B14
:1029B0000299C31A5A1E814200D81A00A04B1A600D
:1029C000904B19681E2353439E4A9B18CB618AE79C
:1029D00001F046FA80239C4ADB02116803900B4306
:1029E00013602268934B994F1A40282313432360A6
:1029F000032001F01DFA03203D6801F019FA3B683D
:102A00000320DB03DB0B009301F012FA3B68ED03BC
:102A1000DB03ED0BDB0B8E4A0193AB18C22B30D8D6
:102A2000009B9B18C22B2CD8019B9B18C22B28D82B
:102A3000009B2A009D4200D21A00009B9D4200D9B3
:102A40001D00019B934200D21300019A954200D9C8
:102A500015005B1B122B14D80C22336814209343EF
:102A6000336033687B4A1340336001F0E1F9082199
:102A70003B682268DB038A432260774ADB0B1360E2
:102A80007FE7032001F0D4F93B68DB03DB0B059300
:102A900001F0E6F9039B0399C21A531E814200D844
:102AA00013006E4A93421BD9FF23356869492D0AEA
:102AB0001D4032686B1C1B060A401B0C134333601D
:102AC0000C23326800209A43083B1343336001F023
:102AD000A7F96348634BA840984206DCFEF732FF33
:102AE000019B009D0093059B95E75F48F6E7002357
:102AF0005E4F554A3B6080231168DB020B43136035
:102B000080222B68032013432B6001F091F93B686E
:102B1000052601333B6080232A685B0213432B6048
:102B20002268444B03201A40514B1343236001F0A9
:102B30007FF90821454B1A682368D2038B43236031
:102B4000454B023900931B68D20B4B439A420CD879
:102B50009B1A3B2B0BD8236846490B4023602B68FC
:102B60000B402B60444B1A601FE7D31AF1E7013E7C
:102B7000F6B2002ED4D123683E4A134023602B685E
:102B800013402B603B68042B07D9BFF34F8F3B4B9F
:102B90003B4ADA60BFF34F8FFEE780222B680320A9
:102BA00093432B6001F044F92268224B03201A4022
:102BB00028231343236001F03BF9244B009A1B6840
:102BC000DB03DB0B1360082223689343236097E742
:102BD00007222C4D2B681340012B02D1002001F05D
:102BE000C7FAAB68284A02201340AB6001F020F915
:102BF0008023AA685B001343AB60D6E64A0AFF1F36
:102C00005CF00040B865FF1F000003400180063DF6
:102C1000BC00034034080000A4000340710200001F
:102C200014100040FFFF3F002810004000E100E0CA
:102C30003075000000FEFEFFC4F0004044F000408C
:102C4000A065FF1F7206000040F0004064F00040E5
:102C500091FCFFFFFF00FFFFA865FF1FE30C0000D2
:102C6000E88000005F361E0060361E002844FF1F0B
:102C700028000100FFFFFEFFA465FF1F00ED00E03C
:102C80000400FA053CF00040FFFEFFFF694E336888
:102C900088331B6883F3088801F02AF900F0C4FB2D
:102CA000654B664A1B68934207D0002001F0B8F8D4
:102CB0000221634A13688B431360FFF703FE614BE5
:102CC000614C1878C0B201F063F90023A3600233AD
:102CD000A3605E4B0120236001F0AAF80323A360E8
:102CE00001F0BEF8040001F0B3F8050001F0B8F8F7
:102CF000574B186001F0CCF8564B1968621A531EF6
:102D0000A14200D213008022D203934201D39B023E
:102D10009B0A3268D16AC90700D478E04E491C0C7E
:102D200009689BB24C4359432402090A64180327DB
:102D30004A49FC3293680A6849489B1A494A4A4EF4
:102D400012684A499B18414A34609A183B400193E3
:102D5000036892089C46019B0A6063440360042B4D
:102D600003D901323B400A6003600B684049E41814
:102D7000200000F0E5FF3F4F3D493B68C3183B6032
:102D80002000019301F034F93B4C206808183849C1
:102D90002060884205D9019B01333B6001F028F98E
:102DA000216000F0EDFF354B1B78002B0ED001F0B9
:102DB0004FF83168324B4A1B1B6812189A4233D2C3
:102DC000591A4919091A2F4801F04AF92E4C237A49
:102DD000002B0FD001F03CF83168E3684A1B121851
:102DE000934224D9591A4919091A284801F038F987
:102DF00000232372264B83F3088801F0C9F90220CF
:102E000000F0C6FF002001F00BF801F0D9F8DC015A
:102E100099000234641A5900641A09214B43803323
:102E2000CB40A408E41882E7FA218900CBE71949CE
:102E3000DBE7C046B865FF1F0C0AFF1FB641210340
:102E400010000040490AFF1F14100040C409000090
:102E5000100AFF1F340AFF1F380AFF1F200AFF1F36
:102E6000280AFF1F1C0AFF1F9C65FF1F240AFF1F63
:102E7000710200006008FF1F2C0AFF1F1C09FF1FC2
:102E8000E408FF1F00100040740BFF1F3C100040BF
:102E900000000020DC050000A022054B92009B589A
:102EA00010B5002B01D0984710BD00F0A9FFFBE73B
:102EB0000000FF1FA122054B92009B5810B5002B6C
:102EC00001D0984710BD00F09BFFFBE70000FF1FFB
:102ED000A222054B92009B5810B5002B01D09847B9
:102EE00010BD00F08DFFFBE70000FF1FA322054B84
:102EF00092009B5810B5002B01D0984710BD00F0F0
:102F00007FFFFBE70000FF1FA422054B92009B58A8
:102F100010B5002B01D0984710BD00F071FFFBE702
:102F20000000FF1F70B500F093FF514B18600420A4
:102F300000F02EFF00F044FF0400C30702D400F0AD
:102F40009FFF70BD00224B4B1A604B4B1878013825
:102F500004282CD800F080FE03231B1F270020002C
:102F600000F036FF0128ECD0444C2378042B71D1BB
:102F700000F096FF002806D001F012F8582001F06A
:102F80002FF802232370032000F002FFD9E720006E
:102F900000F0B6FFE6E7200000F08AFFE2E720003D
:102FA00001F056F8DEE7200000F0B2FEDAE700F0AC
:102FB000CFFF0500012808D1314B1B78053B012BC1
:102FC00003D82000FFF768FFCEE72C4B1B78022BBD
:102FD00001D0052B20D1022D28D12A4B9B7BAB435E
:102FE0001CD12000FFF766FF254B18780128BBD1C4
:102FF0006405B9D4234925224B7B034205D1233AEA
:1030000013405A42534126331A000B7D9342ABD9E9
:10301000322000F09DFEA7E7022D07D1184B1B7848
:10302000052B11D12000FFF753FFDDE7012D0BD158
:10303000012B03D12000FFF759FF95E7062B03D1A1
:103040002000FFF761FF8FE7200000F0D9FE022D7E
:103050008AD1C9E7032B04D10B4B987C00F088FE82
:1030600091E7072B8FD1094B987B00F021FE8AE76F
:103070009C09FF1F9809FF1F9009FF1F2309FF1FCD
:103080001C09FF1FA60BFF1FBC0BFF1FD40BFF1F4C
:10309000FA210A4B0A4A49001A640A4A5A500A4A53
:1030A00004395A50094A08319A64094A5A50094A5F
:1030B0005C315A50084ADA667047C0460000FF1F6C
:1030C0007527FF1F7128FF1F2528FF1F7D23FF1F66
:1030D000E526FF1F011EFF1FD51DFF1F10B500F0C5
:1030E000A3FD10BD8023F7B59C46264B264F0193C8
:1030F0002649274A274D284C284B02281AD16046DA
:1031000038600868264E3040802636033043086019
:1031100001990978002909D11660224A2A60224AB9
:103120002260E02219689143A03A1BE08021C90285
:103130001160F2E766463E600F68194E3E408027F8
:10314000FF023E430E600199097800290DD11760F6
:1031500001280ED1154A2A60154A2260E02219681A
:103160009143C03A0A431A60F7BD80218902116079
:10317000EEE7E0210F4A02432A600F4A22601A68F4
:103180008A43F0E74B0AFF1FE0000340D8000340EA
:103190009000034000000340500003404000034003
:1031A000FFFFE3FF0280063D804508220180063DC7
:1031B000806608220080069880550822F8B51E4BCC
:1031C00080261A68002014003440324232D11A6836
:1031D0001A4F32431A6001223B68063093433B602A
:1031E00000F026FE0122164D2B681E432E603B6820
:1031F0000A2613433B608027BF00124B1B683B42EB
:1032000011D1013EF6B2FF2E09D17E220E4B1C6871
:103210002B68E40B1440934323432B6005E0082004
:1032200000F006FEE9E7002EEFD180222B6860084F
:1032300093432B60F8BDC046C4F000405CF00040F2
:1032400018F0004068F0004060F0004010B500F059
:1032500037FE01215820034A00F0D2FEFFF7AEFFEF
:1032600010BDC046600AFF1F10B578220021034838
:1032700000F02EFF00F0CCFE002010BDC068FF1F44
:1032800070B5040000F02CFE00230C200B4A010056
:1032900059438D18515C00290DD0A14208D101235A
:1032A00000246B7000F05CFF00F0EAFE200070BDAF
:1032B00001330A2BEBD11224F6E7C046C068FF1F8A
:1032C00070B5040000F00CFE002319001D000D4A2B
:1032D0001078002806D0A0420CD1557001310C3274
:1032E0000A29F5D1002B0AD100F092FE00F0C8FEA9
:1032F000002070BD5078461EB0411B18EEE700F06C
:103300002FFFF3E7C068FF1FF7B504000C20002370
:1033100084460E4D019267465F43E85D7E19A042E8
:1033200012D000280BD10A4B9C4662461B7808330A
:103330001370019B70707C557160B360FEBD0133EA
:103340000A2BE8D10320F9E70720F7E7C068FF1F41
:10335000BC68FF1F8021204BC9051B6870B58B60BE
:103360001E4BC1241A680123FF2013434B611C4BE1
:10337000A4001A681B4B00251A601B4B1A681B4BD4
:103380001A601B4B1A5982431A51C52292009C584D
:103390008443BF38204398509C58164804408020EE
:1033A000C001204398509858134C0002000A014372
:1033B0009950124B1B78DB08AB4201DC002070BD3A
:1033C0002378002B06D0A368002B00D09847013546
:1033D0000C34EEE71220F2E7C044FF1FBC44FF1F8D
:1033E000B0F00040B868FF1FB4F00040B468FF1FA1
:1033F00000E100E0FF00FFFFC068FF1FBC68FF1F87
:10340000030010B51F2809D8072200201340072405
:1034100004490A78A24313430B7010BD0023062011
:10342000F5E7C046BC68FF1F034A04491368002043
:103430000B4013607047C0461CF00040FFFFC1FF07
:10344000054B06491B780A6805485B0702401B0BC1
:10345000134300200B607047BC68FF1F1CF0004046
:10346000FFFFC1FF70B50C25FFF7EAFF0A4B1C7880
:103470000A4BE4086543ED18002C01D1200070BD13
:103480002B78002B06D06B68002B00D09847013CAE
:103490000C3DF1E71220F2E7BC68FF1FB468FF1F84
:1034A00007B50422074801A900F034F9019B013354
:1034B00005D18023044ADB0411680B43136000200C
:1034C0000EBDC0461C18001114F00040F0B50500F8
:1034D0002026184B87B00493049B002B03D11124A2
:1034E000200007B0F0BD002102220B0001910091E5
:1034F000052000F045FD02230F490A681A42FCD15D
:103500000596059C631E0593002CFAD10B4A13689F
:10351000002BFCDA0F276F440121380000F0C8FDB2
:103520003B782B42DCD0052000F082FC049B013B61
:103530000493D1E7FFFFFF0790C8004000C8004098
:1035400007B500F0CDFC80220821D205936A0191D5
:10355000002B01D10739916202210C4A11600199B7
:10356000481E01900029FAD1033111600531019103
:103570000199481E01900029FAD11160002B02D157
:103580008022D205936200F07BFD07BD00C00040A1
:10359000F0B52D4C89B02378002B4FD1FEF7B2F94E
:1035A00002232A4F03903A681A42FCD12023069343
:1035B000069B5A1E0692002BFAD1254E3368002B2B
:1035C000FCDA0120FFF782FF011E02D0112009B0B2
:1035D000F0BD030003220190009005AD9F2000F094
:1035E000CFFC0321280000F063FD02233A681A4251
:1035F000FCD120230793079B5A1E0792002BFAD178
:103600003368002BFCDA0120FFF760FF0028DDD1D2
:103610000398FEF78BF9AA786B7811041B020B4311
:1036200029780B4363601300113B0A49052B07D827
:1036300001239340A3600B60012323700020C6E7A1
:1036400080231B03F6E7C046A844FF1F90C8004034
:1036500000C800409808FF1F1E4B30B55A68187804
:103660001D4B85B0D31859424B41012100930023D3
:1036700000F0FEFB194B1A4A02259A6300221A65D4
:1036800010325A658022C4219D65164B1648D2021D
:10369000DA6789004258154B80241A4080231B04A6
:1036A00013434350642341200393E40500F078F969
:1036B000402000F075F96562039D6B1E0393002D99
:1036C000FAD103236362FFF73BFFA562FFF760FFB8
:1036D00005B030BDB444FF1F95FFFEF700C80040A1
:1036E000050001FF04E100E000E100E0FFFF00FF52
:1036F00010B5064B18705960FFF7AEFF002113207C
:10370000034AFFF701FE002010BDC046B444FF1F6E
:103710005936FF1FF0B5040085B003920291FEF701
:10372000F1F8882263035B0B52051A438023DB0503
:103730009D6A8023274F0092BA68002601901B03E0
:103740009A420CD9F82326001B041E401C4206D0C6
:103750008022214B52025E6219680A431A60002DD2
:103760000BD100F0BDFB02221C4B1A608023DB054D
:103770005A62013A9A6200F083FC0023039A934252
:1037800020D1002D0AD100F0ABFB144B03221D60A9
:103790008023DB055A629D6200F072FC8023BA68C8
:1037A0001B039A4208D9002E06D000220A4B0C496E
:1037B0005A621A680A401A600198FEF7B7F80020AA
:1037C00005B0F0BD009A0299D2181278CA5401339C
:1037D000D4E7C046A844FF1F00C8004000C0004016
:1037E000FFFFFEFFF0B587B0029103920400FEF7E1
:1037F00089F8019000F074FB802302250122234EFA
:10380000DB0535605D629A6200F03AFC204F3B6850
:103810002B42FCD120230493049B5A1E0492002BBC
:10382000FAD11C4D2B68002BFCDA0120FFF74EFE6D
:10383000002802D0112007B0F0BD2000039A0299A1
:1038400000F086FC022304003A681A42FCD12023CF
:103850000593059B5A1E0592002BFAD12B68002B6D
:10386000FCDA0120FFF732FE051EE3D100F038FB41
:1038700080230322DB0535605A629D6200F000FC64
:103880000198FEF753F8E0B2D5E7C04600C000400B
:1038900090C8004000C80040F0B5802687B0040002
:1038A000FEF730F8F605B36A02250393029000F0A4
:1038B00017FB0123244F3D607562B36200F0E0FB0B
:1038C000224E33682B42FCD120230493049B5A1EC2
:1038D0000492002BFAD11E4D2B68002BFCDA01203C
:1038E000FFF7F4FD002802D0112007B0F0BD200042
:1038F00000F0E6F90223019032681A42FCD120233D
:103900000593059B5A1E0592002BFAD12B68002BBC
:10391000FCDA0320FFF7DAFD041EE5D100F0E0FA3F
:1039200080230322DB053C605A629C6200F0A8FB06
:10393000039B002B01D1FFF703FE0298FDF7F6FF72
:103940006B461879D1E7C04600C0004090C80040DF
:1039500000C8004007B5000201910422000A01A935
:10396000FFF740FF0EBD000073B5050005240B4AAC
:10397000A3005B429B1819686B46DE1D300000F007
:10398000AFFB022804D133782B55013CEFD276BD32
:10399000052CFCD00128FAD10230F8E714090011F7
:1039A0001F2807D8012380228340D20591680B434A
:1039B000936070473F2808D8012380222038834035
:1039C000D20551690B435361F3E75F28F1D8012316
:1039D000802240388340D205116A0B431362E8E726
:1039E0001F2807D8012280218240C9058B68934394
:1039F0008B6070473F2808D8012280212038824000
:103A0000C9054B6993434B61F3E75F28F1D8012265
:103A1000802140388240C9050B6A93430B62E8E776
:103A20001F2810D880230200DB05153A1968012AE7
:103A300006D820229143196019680A431A6070471A
:103A400001228240F6E73F2811D880230200DB05DF
:103A5000353AD968032A06D810229143D960D9682B
:103A60000A43DA60EBE7012220388240F5E75F285D
:103A7000E5D842238022181A413B8340D205516A7F
:103A800099435162516A0B435362D8E710B5040061
:103A9000012813D1A022184992050B685B015B092C
:103AA00013430B60154B164A19681140154A0A4317
:103AB0001A60402219680A431A6010BD0028FCD120
:103AC00001000A2000F084FA21000B2000F080FAA7
:103AD000C0220A4B920019680A4340211A601A68F2
:103AE0008A431A60B022044912060B685B015B0925
:103AF00013430B60E1E7C04614F000401CF00040A7
:103B00007F00FEFF80FD0100FA2110B58900C0038F
:103B100000F016F900F08CF910BD000072B6074AEB
:103B20001368013313600422054B1A600023054A11
:103B300013608022D2055360FEE7C0467808FF1F5D
:103B4000C0F00040C4F00040044B054A1A60054B29
:103B50001A600022044B1A607047C046140AFF1F07
:103B6000841E0000380AFF1FC4F000400023034AEF
:103B70001360034A1360034A1360704754F0004017
:103B800040F1004044F10040002310B5184C8AB0C9
:103B9000009301932378012B27D06946012000F080
:103BA0000FFB002817D1009B12490293019B06AA24
:103BB0000393114B02A81B680493104B1B680593D9
:103BC00000F086F910220E4906A800F061FA0028DC
:103BD00004D1FF23237000200AB010BD0123094A3D
:103BE000074902A8237000F073F90120F4E7C046EA
:103BF000BC65FF1F10290011082900110C290011B4
:103C000020290011C065FF1F13B50124694601205A
:103C100000F0D6FA034B00940193FFF7B5FF2000A4
:103C200016BDC046BB0B000010B5FFF79FFFFFF7A6
:103C3000EBFF002802D0024B984710BDFEE7C046BC
:103C4000E1A2000002B47146490849000956490042
:103C50008E4402BC7047C04602B471464908490010
:103C6000095C49008E4402BC7047C04603B47146EB
:103C7000490840004900095A49008E4403BC704776
:103C800001B40248844601BC604700BF69110100CD
:103C900001B40248844601BC604700BFE927000028
:103CA00001B40248844601BC604700BF71B0000007
:103CB00001B40248844601BC604700BFC1F7000060
:103CC00001B40248844601BC604700BFA96F0100EF
:103CD00001B40248844601BC604700BFE9D400003B
:103CE00001B40248844601BC604700BFE94C0100B2
:103CF00001B40248844601BC604700BFC1A5000072
:103D000001B40248844601BC604700BF8937010006
:103D100001B40248844601BC604700BFF935010088
:103D200001B40248844601BC604700BF851201000F
:103D300001B40248844601BC604700BFF9A60000F8
:103D400001B40248844601BC604700BF090E000070
:103D500001B40248844601BC604700BF61370100DE
:103D600001B40248844601BC604700BFE90B010072
:103D700001B40248844601BC604700BF4DF9000011
:103D800001B40248844601BC604700BFD54401002D
:103D900001B40248844601BC604700BF1907010016
:103DA00001B40248844601BC604700BF8D82000018
:103DB00001B40248844601BC604700BFA9D8000096
:103DC00001B40248844601BC604700BFBD0B01003E
:103DD00001B40248844601BC604700BF01340100C1
:103DE00001B40248844601BC604700BFA1AF000097
:103DF00001B40248844601BC604700BF8B520100F9
:103E000001B40248844601BC604700BFE9170100C5
:103E100001B40248844601BC604700BFB3520100B0
:103E200001B40248844601BC604700BF016C010038
:103E300001B40248844601BC604700BF018900000C
:103E400001B40248844601BC604700BF6D0B01000D
:103E500001B40248844601BC604700BFC95C010050
:103E600001B40248844601BC604700BF156B0100E5
:103E700001B40248844601BC604700BFC56D010023
:103E800001B40248844601BC604700BFDD0A01005E
:103E900001B40248844601BC604700BFC16601000E
:103EA00001B40248844601BC604700BF01D700004E
:103EB00001B40248844601BC604700BF05340100DC
:103EC00001B40248844601BC604700BFED680100B0
:103ED00001B40248844601BC604700BFDD3F0000DA
:103EE00001B40248844601BC604700BF75A90000C8
:103EF00001B40248844601BC604700BFC9A9000064
:103F000001B40248844601BC604700BF0934010087
:103F100001B40248844601BC604700BFF90D0100AE
:103F200001B40248844601BC604700BF116E000026
:103F300001B40248844601BC604700BF9D6A00008E
:103F400001B40248844601BC604700BFF9ED00009F
:103F500001B40248844601BC604700BFDD0C01008B
:103F600001B40248844601BC604700BFE9F6000086
:103F700001B40248844601BC604700BFCD0C01007B
:103F800001B40248844601BC604700BF496D01008E
:103F900001B40248844601BC604700BF8914010097
:103FA00001B40248844601BC604700BF6DF60000C2
:103FB00001B40248844601BC604700BFBD5C0100FB
:103FC00001B40248844601BC604700BF855201002D
:103FD00001B40248844601BC604700BFF999001152
:103FE00001B40248844601BC604700BF7912010059
:103FF00001B40248844601BC604700BF090E0000BE
:1040000001B40248844601BC604700BF016701005B
:1040100001B40248844601BC604700BFADAE000059
:1040200001B40248844601BC604700BF53B9000098
:1040300001B40248844601BC604700BF59760100C4
:1040400001B40248844601BC604700BFE51201008C
:1040500001B40248844601BC604700BFF535010049
:1040600001B40248844601BC604700BF2D6C0100CA
:1040700001B40248844601BC604700BF8D110100B5
:1040800001B40248844601BC604700BF9DA90000FE
:1040900001B40248844601BC604700BFCD4C01001A
:1040A00001B40248844601BC604700BF0D520100C4
:1040B00001B40248844601BC604700BF3D71010065
:1040C00001B40248844601BC604700BF85C10000BE
:1040D00001B40248844601BC604700BFB70E00002F
:1040E00001B40248844601BC604700BF2D3800116E
:1040F00001B40248844601BC604700BFED6B01007B
:1041000001B40248844601BC604700BF75F8000056
:1041100001B40248844601BC604700BF09AE0011EB
:1041200001B40248844601BC604700BF19FA000090
:1041300001B40248844601BC604700BFC1150100BC
:1041400001B40248844601BC604700BFD9B00000FA
:1041500001B40248844601BC604700BF957301006A
:1041600001B40248844601BC604700BF21A9000099
:1041700001B40248844601BC604700BFEDA50000C1
:1041800001B40248844601BC604700BF8944000076
:1041900001B40248844601BC604700BF7997000023
:1041A00001B40248844601BC604700BF51B800001A
:1041B00001B40248844601BC604700BF21440000AE
:1041C00001B40248844601BC604700BFE1AC000076
:1041D000020000002AB700110100000010B5001114
:1041E0000200000026B70011010000001042FF1F6E
:1041F0000200000018B50011010000001863FF1F45
:104200000200000024B70011030000008C62FF1FB1
:1042100012000000020000002AB700110100000097
:1042200058B500110200000026B70011010000007F
:1042300055B500110200000062B500110300000036
:10424000C762FF1F0200000024B700110300000036
:10425000DC62FF1F0200000026B700110100000011
:1042600054B500110200000060B500110300000009
:104270009D62FF1F0200000024B700110300000030
:10428000BE62FF1F020000002AB7001101000000FB
:104290009CB500110200000026B7001101000000CB
:1042A0005943FF1F02000000AEB5001101000000DD
:1042B00093B500110200000026B7001101000000B4
:1042C0005843FF1F02000000ACB5001101000000C0
:1042D000E462FF1F0200000026B700110100000089
:1042E0005743FF1F02000000AAB5001101000000A3
:1042F00083B500110200000026B700110100000084
:104300005643FF1F02000000A8B500110100000085
:104310007EB500110200000026B700110100000068
:104320005543FF1F02000000A6B500110100000068
:1043300079B500110200000026B70011010000004D
:104340005443FF1F02000000A4B50011010000004B
:1043500074B500110202020202020000C9470011F6
:10436000C5470011D8B5001190011D0018001800B4
:10437000FFFF07010203040506020106000000001A
:10438000000000000000000000000000000000002D
:104390000000000000000000030000000200000018
:1043A0002AB700110100000058B6001102000000F9
:1043B00026B70011010000000C44FF1F020000009E
:1043C00062B60011010000001263FF1F020000002E
:1043D00024B70011030000006C65FF1F02000000FD
:1043E00026B70011010000000C44FF1F020000006E
:1043F00060B60011010000001463FF1F02000000FE
:1044000024B70011030000006465FF1F12000000C4
:104410000001000000000111FFFF00005048593664
:10442000000000000000000001000000E9B50011DC
:104430000B000500F7000000B40000280028002849
:104440003075A000A000A000A00000080008E00156
:10445000F0001000100010001000100010005000BC
:104460005000500010001000D007000000000000B5
:104470000F0001000500307507001000010081FFEA
:1044800000000000FF000000F16B0011F96900114D
:1044900089670011FFFF0100FF000000ED9500118A
:1044A00069930011819200110000000000000000DB
:1044B00000000800040000003B0001085902E00170
:1044C00088212800FF000000020000002AB7001128
:1044D00001000000F0B700110200000026B7001133
:1044E000010000004545FF1F0200000022B7001137
:1044F000010000007869FF1F0200000026B70011CC
:10450000010000004445FF1F0200000020B7001119
:10451000010000004245FF1F0200000026B7001105
:10452000010000004045FF1F020000001EB70011FF
:10453000010000003845FF1F180018001D00900101
:104540000200000302020000020000002AB700116E
:104550000100000004B800110200000026B700119D
:10456000010000008845FF1F020000001CB7001179
:1045700000000000000000000200000024B700114D
:0A458000030000009869FF1F20FFF0
:040000051FFF184180
:00000001FF
